:020000040000FA
:0600000095EF3BF0120039
:06000800BEEF00F0120043
:06002A00010076770000E2
:08003000800000007B000000CD
:04017C00DACFE4FFF3
:10018000E2CFDAFFE9CFE4FFEACFE4FFF3CFE4FF09
:10019000F4CFE4FF00EE00F0180EE80403E3EECF26
:1001A000E4FFFBD7E652F2A402D035D8F2949EA029
:1001B00002D032D89E909EA202D02FD89E92A1A2A9
:1001C00002D041D8A1929EA402D0C8D89E94A1A0EA
:1001D00002D0E9D8A1909EAA02D00BD99E9A9EB8CF
:1001E0009E98F2B2F292F0B0F090F0B2F092E55236
:1001F00000EE17F0180EE80403E3E5CFEDFFFBD7A0
:10020000E5CFF4FFE5CFF3FFE5CFEAFFE5CFE9FF68
:10021000E5CFDAFF1100120012000101BE71BE51DC
:10022000EA6ABF0FE96E010EEA22EF50CB6EBE05FF
:1002300004E18280010EE66E02D08290E66A93ECC1
:100240000FF0E55212005BEC21F0050EE126950E51
:10025000E66EE70EE66ED3EC3AF0E552E552D95081
:10026000010F53EC24F0030F5AEC24F0ED6E010162
:100270006251622B0D0805E26B0502E0010E6B6F07
:10028000626BFF0E575D01E2572B680526E157515F
:1002900062083FE23CEC26F008E1EE507A1905E1F5
:1002A000EE507B1902E1EE507C190AE093EC22F04B
:1002B000EA0EEE6E030EED6EB0EC23F0EA0E03D004
:1002C00000EC29F0E80EEE6E030EED6EB66BB76B28
:1002D000B86BB96B58051DE01AD05751060819E2E2
:1002E0003CEC26F00EE1EE507A190BE1EE507B1952
:1002F00008E1EE507C1905E104E100EC29F0AAECDC
:1003000026F0B66BB76BB86BB96B580502E0010EFF
:10031000586F3FEC29F009E1030EED1806E10A0ED3
:10032000A627000EA723A823A923030EB0EC23F0D1
:10033000E90EEE1809E1030EED1806E10A0EAE27EC
:10034000000EAF23B023B123C80506E10A0ECF2764
:10035000000ED023D123D22342EF21F0BEEC28F0AF
:100360000101680508E174EC1AF0850EAFEC26F087
:100370000101686B0CD0580502E1066B02D081ECDC
:100380001AF0840EAFEC26F00101010E686F000E2A
:10039000E66EE66AE9EC3AF0E552E5520101576B88
:1003A000586B42EF21F0020E0101735D0AE1020E6B
:1003B0007927000E7A237B237C23020E8127000EEF
:1003C00014D0080E735D0FE10001F80509E1010189
:1003D00043EC26F08223832384230001F86B120070
:1003E000010EF86F120043EC26F08223832384234E
:1003F00012008AEC27F0A1EC3AF0DF6E020EDF5C0F
:1004000003E10101020E0BD0060EDF5C03E10101E6
:10041000060E05D0150EDF5C03E10101150E726FAB
:1004200088EF22F0EFD801D9AFEC0FF00101006F97
:10043000C2EC0FF0809630EC21F00101736FA2EC5A
:1004400010F0020A03E0020A04E103D026EC20F0D7
:1004500001D002D801EF03F0D9CFE6FFE1CFD9FFF9
:10046000050EE126A8EC0BF073EC19F0BAEC19F0CC
:10047000CAEC19F0EDEC19F0030EDB68010161051F
:1004800005E1C4EC1AF00101616BB4D0310E925C4D
:1004900005E1930403E1B60E945C10E0310E926E18
:1004A000010E936EB60E946E070EE66EAE0EE66EFD
:1004B0004BEC3AF0E552E5529DD009D00F0EC11435
:1004C0000E0805E0F00EC1140E09C16E93D00101B3
:1004D0006B0509E10101765106E1030EDB6A47EC89
:1004E0000BF001016B6B01016B0516E1020E0101BE
:1004F000765D12E1460E006E01017851D8800054FD
:100500000BE301017851470807E3020EF36E030E77
:10051000F3CFDBFF01016B6BA2EC10F0DF6EDF505D
:1005200039E0FF0EDF5C36E0010EDB50DF5C16E1E8
:10053000030EDF5C03E0040EDF5C10E101016C518F
:100540000CE1140E006E040EDB2A040EDB50D88082
:10055000005403E30101010E6C6F03D0010EDFCFE5
:10056000DBFF020EDB5003E001016C0512E1030E1C
:10057000DB50FF080EE1DFCFE6FF37EC11F0E5526C
:10058000E76E030EE7CFDBFF010EF36E020EF3CF33
:10059000DBFF0BD0DF5009E1020EDB6A010EDB6AE4
:1005A000040EDB6A01016C6B00D0030EDB50FF0808
:1005B00006E0030EDBCFE6FFA5D8E5521BD028EC02
:1005C00010F05FEC10F000090BE07BEC10F07AEC1F
:1005D00010F00300000090EC10F069EC18F00AD065
:1005E000070EE66EAE0EE66E4BEC3AF0E552E552C3
:1005F00001D044D741D7D9CFE1FFE552E7CFD9FFAA
:100600001200FFD74AEC26F0806A816A826A8EEC7B
:1006100025F00F0EE66EE66A2C0EE66EF9EC39F068
:10062000E552E552E5521DEF25F0010ED8EC25F01C
:10063000020ED8EC25F00101100E916F270E926F7B
:10064000960E936F500E946F19EC25F0DE0EE66E49
:10065000000EE66EB60EE66E010ED4EC27F055ECF9
:1006600028F0070EE66EE66AE20EE66E000EE66E13
:10067000BA0EE66E010ED4EC27F027EC25F0D4EC90
:1006800027F00101626B766B756B776978696B6B2C
:10069000716B6E6B616B010E686F576B586B829656
:1006A0001200C3EC28F0DF6A080EDF5C29E2DF509D
:1006B000080DF3504009E66E62EC37F0E552010E8A
:1006C000DB6A080EC8EC28F019E2DF50080D16ECC2
:1006D00028F0BD0E00266D0E0122010EDB500F0129
:1006E0000024F66F000E0120F76F0800F550E66E4B
:1006F00055EC37F0E552010EDB2AE3D7DF2AD4D7D9
:1007000042EF21F05BEC21F0FE0EDB5002E114D849
:1007100011D0FE0EDB0404E10101BD6B82D80AD0CA
:10072000FE0EDB50020802E1EDD804D0D7EC26F033
:1007300001E124DA82EF27F0BEEC28F001017551C7
:1007400002E0750508E1D950010FEBEC26F0890EA7
:10075000EE6E010E0AD0020E755D03E0030E755DAC
:1007600005E1D950010F5AEC24F0ED6E6E5101E015
:100770006E07755103E0020E755D1CE16E5105E0D8
:10078000010EE66EEDEC0EF010D03FEC29F00AE120
:10079000030EED1807E19E5105E0010EE66E61ECD7
:1007A0000AF003D0010EE66ED3DAE552020EE66ED1
:1007B00094DB2ED0750503E0030E755D1DE16E51CF
:1007C00005E0010EE66EEDEC0EF010D03FEC29F0E6
:1007D0000AE1030EED1807E19E5105E0010EE66EF9
:1007E00061EC0AF003D0010EE66EB2DAE552020EB9
:1007F000E66E0BEC08F00CD0040E755D0BE1010EFB
:10080000E66EECEC08F0E552020EE66E22EC09F022
:10081000E55205D0050E755D02E1C9EC09F042EF25
:1008200021F05BEC21F0250EE126D950230FEBECF3
:1008300026F03A0EEE6EEE6ACF0EE66E6C0EE66EA7
:10084000D950010F87EC21F0CF0EE66E6C0EB4ECA0
:1008500028F0E66ACAEC37F0E5520A0E006E010194
:100860007751005C4DE3006A7751D88000541FE354
:10087000775109081CE37751010B775DB9EC28F03B
:1008800001017751010B02E0000E01D0010E772526
:100890002AEC27F0D950010F86EC27F0010177519F
:1008A000010B110D05EC29F07E0EEF6E1BD0775178
:1008B000010B0DE07705B9EC28F0010177512AEC26
:1008C00027F07E0EF36E120EF3CFDBFF0BD07751C5
:1008D000B9EC28F0A6EC29F0020F9BEC22F0DE52D6
:1008E0007E0EDD6EDF6A020EDF5C0AE2DF288AEC34
:1008F00028F0010F39EC23F08FEC28F0DF2AF3D732
:1009000042EF21F05BEC21F0250E8FEC24F051EC4E
:1009100026F00A0E006E7751005C01E22DD16C05C5
:1009200007E1460E54EC25F003E37851470802E254
:100930007EEC37F0DE525B0EDD6E01017751BEECCE
:1009400021F0020F87EC21F05D0EF36E100EF3CF55
:10095000DBFF110EDB6AFF0E0101785D2BE1F3EC8A
:1009600024F0FF0823E161EC22F0060808E061ECC6
:1009700022F0050804E061EC22F0070802E1640EB1
:1009800011D061EC22F0020802E1660E0BD061EC9E
:1009900022F0030802E1650E05D061EC22F00408A4
:1009A00003E1670E786F06D0786904D0B3EC27F0C6
:1009B000EFCF78F1640E785D09E0650E785D06E0B2
:1009C000660E785D03E0670E785D10E1640E785D79
:1009D000110D16EC28F07A0E00266C0E0CEC29F0A6
:1009E000120FE3EC26F02CEC39F07DD07851006E3C
:1009F000016AFF0E001803E1015001E1BDD0B3EC24
:100A000027F0EE52EFCF00F0F3EC24F00024785DF5
:100A100053E2F3EC24F0785D110DF350026E036A9B
:100A2000230EDBCFE9FF240E28EC24F0D950120F5F
:100A300087EC21F0020E0101785D0BE1D9501A0F0D
:100A4000E3EC26F095C1E6FF96C1E6FF01EC0CF061
:100A50004AD0030E785D05E108EC25F097C1E6FF6A
:100A600007D0040E785D07E108EC25F098C1E6FF99
:100A70000CEC0CF039D00D0E54EC25F00AE3785153
:100A8000100807E3D9501F0FE3EC26F01DEC0FF020
:100A90004DD0110E785D07E1D950120FE3EC26F02E
:100AA0004FEC0FF043D0120E785D42E1D9501C0F8D
:100AB000E3EC26F053DB3AD0330E54EC25F02BE375
:100AC0007851360828E3330E785D10E18A0EE66E21
:100AD0006D0EB4EC28F008EC25F099C1E6FF9AC140
:100AE000E6FF32EC0CF0E552E55220D0340E785D92
:100AF00006E0350E785D03E0360E785D19E19B0E59
:100B0000E66E6D0EB4EC28F0D950190FE3EC26F028
:100B10003BEC0CF00BD0460E54EC25F009E3785179
:100B2000490806E3ACEC29F080EC0CF0E552E55204
:100B3000650E0101785D06E0660E785D03E0670EE4
:100B4000785D05E1DAEC1EF00101030E766FDF6AD5
:100B5000020EDF5C0FE2DF28E66EF2EC21F0B4EC6F
:100B600026F039EC23F089EC37F0E552E552E552F6
:100B7000DF2AEED72CEC0EF042EF21F012005BECF6
:100B800021F00D0EE126000E0101715D14E3640EEB
:100B9000006E7151005C0FE3FBEC26F071C1E6FFC3
:100BA0000C0E02EC24F037EC27F00C0EE66ED9CFD9
:100BB000E6FF23EC23F042EF21F05BEC21F0070E7F
:100BC000E126020EF36EFE0EA1EC22F001E2BED091
:100BD000000EF36EFD0EA1EC22F001E2B7D0640E20
:100BE000006EFD0EDB50005C01E2B0D0FE0EDB506B
:100BF000050DF350FE0FDF6EDF50046E056AFD0E2B
:100C0000DB50026E036A1E6E03C01FF004C023F0A7
:100C100005C024F0A2EC31F01CC000F01DC001F0B2
:100C2000640E236E246A1CC01EF01DC01FF0FFEC72
:100C30003AF01FC001F0010E1EC0DBFFDB5005E1E2
:100C4000020EDB6A030EDB6A29D0010EDB500408BA
:100C500005E3020EDB6A010EDB501CD0010EDBCF78
:100C600000F0040EDF5CD880005407E338EC24F079
:100C7000020EDB50050DF3500BD0010EDBCF00F060
:100C8000DF50D88000540AE338EC24F0030EDF5C18
:100C9000E552E75CE76E030EE7CFDBFF040EDB6A8D
:100CA000FE0EDB50F36E040EA1EC22F04FE2020EBA
:100CB000DB50F36E040EDB50F35C1EE1A3EC28F076
:100CC0001F50F36E040EDB501F5C0AE158EC26F057
:100CD00007E1030EDB28F76A020FF66E6E0E06D0F0
:100CE000030EDB50F76AFD0FF66E6D0EF72208005B
:100CF000060EF5CFDBFF19D058EC26F002E1BA0E54
:100D000008D0020EDB50F36E040EA1EC22F004E2D8
:100D1000070E59EC25F009D0040EDB50F36E020EDD
:100D2000A1EC22F002E2060EDB6A040EDB50E76E55
:100D3000FB0EDBCFE9FFFC0EDBCFEAFF7BEC24F000
:100D4000060EDBCFEFFF040EDB2AAAD742EF21F01D
:100D50005BEC21F02D0EE126D9501E0F5FEC26F042
:100D6000EE6E08EC24F0530EEE6E540EEE6E4F0E47
:100D7000EE6E500E51EC28F0280FEBEC26F0460EEC
:100D8000EE6E430EEE6E550EEE6E540EEE6EEE6A85
:100D9000090EDB6A0101755102E0750508E1D950C1
:100DA0001A0F53EC24F01C0F89EC23F00FD0020E25
:100DB000755D03E0030E755D0AE1D9501A0F5AEC18
:100DC00024F0ED6ED9501C0FE5EC23F0ED6EB8EC7D
:100DD00021F0E80EEE1802E1030EED1810E0B8EC79
:100DE00021F0E90EEE1802E1030EED1808E0B8EC70
:100DF00021F0EA0EEE1806E1030EED1803E1070EEE
:100E0000DB6A2BD0B8EC21F019EC23F0FA0ED88075
:100E10000054000E015404E2640EB9EC26F01DD01B
:100E2000B8EC21F019EC23F0640E0102F3CF01F0CD
:100E30000002F3CF00F0F4500126FA0E236E246A6C
:100E4000F3CF1EF001C01FF0FFEC3AF01EC000F01F
:100E50001FC001F0070E1EC0DBFFD950090FE3ECE5
:100E600026F0070EDBCFE6FF0C0E02EC24F0B8EC08
:100E700021F0E80EEE1806E1030EED1803E1D9505B
:100E80001E0F1DD0B8EC21F0E90EEE1806E1030E9E
:100E9000ED1803E1D950230F12D0B8EC21F0EA0E7F
:100EA000EE1806E1030EED1803E1D950280F07D024
:100EB00064EC26F0B8EC21F0F1EC27F0020FA6EC80
:100EC00021F0150FECEC29F0100EE66ED950090F49
:100ED000E66E23EC23F042EF21F05BEC21F0290ECB
:100EE0000CEC25F06B0EEE6E6D0EEE6E3A0E51ECC4
:100EF00028F0040FEBEC26F04C0EEE6EEE6A140EAA
:100F0000DB6A0101755102E0750508E1D950250F32
:100F100053EC24F0270F89EC23F00FD0020E755DFF
:100F200003E0030E755D0AE1D950250F5AEC24F059
:100F3000ED6ED950270FE5EC23F0ED6ED9500D0F73
:100F4000E3EC26F0270EDBCFE9FF280EDBCFEAFF2C
:100F500032EC24F0D950060FE3EC26F00D0EDBCF77
:100F6000E6FF0E0ECEEC27F0070FA6EC21F0140FD3
:100F70004CEC21F02E0EF36E180EF3CFDBFFE66A79
:100F8000D950060FE3EC26F00F0EDBCFE6FF100E74
:100F9000CEEC27F0070FA6EC21F0190F4CEC21F056
:100FA000190EDB50200805E1300EF36E190EF3CF59
:100FB000DBFFFBEC26F0D9501A0F4CEC21F0250E8C
:100FC000DBCFE9FF260EDBCFEAFF120EEECFDBFF11
:100FD000130EEDCFDBFFDBEC26F0060FE3EC26F083
:100FE000120EDBCFE6FF130ECEEC27F0060FA6ECB9
:100FF00021F01D0F21EC28F0040FA6EC21F0230FA7
:10100000ECEC29F0100EE66ED950140FE66E23ECCE
:1010100023F042EF21F05BEC21F03B0E0CEC25F0CD
:10102000CD0EEE6EB20EEE6EB70EEE6EDD0EEE6E05
:10103000C80EEE6EDD0EEE6ECB0EEE6EDF0E8BEC9E
:1010400022F0EE6AD950110FEBEC26F06B0EEE6E2B
:101050006D0EEE6EEE6A280EDB6AFBEC26F0D950C0
:10106000280F4CEC21F00101755102E0750505E1F6
:10107000D950390F89EC23F00AD0020E755D03E0D8
:10108000030E755D05E1D950390FE5EC23F0ED6EE7
:1010900068EC26F071EC25F0170EEECFDBFFFEECCE
:1010A00024F068EC26F044EC29F0180E1CC0DBFF9D
:1010B000190E1DC0DBFF1A0E1EC0DBFF1B0E1FC06A
:1010C000DBFF140EDBCF04F0150EDBCF05F0160EA0
:1010D000DBCF06F0170EB7EC29F0800E0C6EA60ED3
:1010E0000D6E3F0E0E6E910E0F6E180EDBCF14F0CC
:1010F000190EDBCF15F01A0EDBCF16F01B0EDBCF6F
:1011000017F014C01CF015C01DF016C01EF017C05B
:101110001FF015EC22F01F0E1EC0DBFF200E1FC0BB
:10112000DBFFDBEC26F0210FE3EC26F01F0EDBCF1C
:10113000E6FF200ECEEC27F0220FA6EC21F0310FB7
:1011400021EC28F0110FA6EC21F0360FECEC29F081
:10115000D950280FE6EC22F042EF21F05BEC21F0B1
:10116000080EE126010EDB6A020EDB6A010EBEEC00
:1011700026F0060EDDEC25F0DF6A040EDF5C0DE2E2
:10118000D950010F48EC29F0A6EC22F0010FDDEC5C
:1011900029F06EEC29F0DF2AF0D7040EDB50E76E61
:1011A000050EE7CFDBFF030EDB50E76E040EE7CF43
:1011B000DBFF2E0EBEEC26F0200E59EC25F0070EBC
:1011C000DB6A010EDB50300803E1DE52200EDD6EDB
:1011D000D950010F27EF2AF05BEC21F0200EE12619
:1011E000D950030FEBEC26F0530EEE6E700EEE6E40
:1011F0006C0EEE6E730E8BEC22F0EE6E5B0EEE6EEE
:10120000500EC0EC25F01E0F4BEC29F0140FE3EC50
:1012100026F01E0EDBCFE9FF1F0EDBCFEAFF41EC0D
:1012200024F0080EACEC23F0160FA6EC21F0080F0A
:10123000B0EC29F037EC27F0D950030FE6EC22F0A0
:1012400042EF21F05BEC21F0300E6FEC26F0460E01
:10125000EE6E4C0E8BEC22F0EE6EEE6EEE6EEE6EDF
:10126000EE6EE7EC25F02E0E08EC24F04C0E5EEC52
:1012700025F0050EF36E260EF3CFDBFF070EF36E9F
:10128000270EF3CFDBFF080EF36E280EF3CFDBFF44
:10129000090EF36E290EF3CFDBFF0A0EF36E2A0E52
:1012A000F3CFDBFF0B0EF36E2B0EF3CFDBFF0C0E39
:1012B000F36E2C0EF3CFDBFF0D0EF36E2D0EDFEC75
:1012C00026F02E0F89EC23F0ED6EFEEC24F02E0EAE
:1012D000DBCFE9FF2F0EDBCFEAFF44EC29F0020E53
:1012E0001CC0DBFF030E1DC0DBFF040E1EC0DBFFB6
:1012F000050E1FC0DBFFD950170FA6EC21F0020F1F
:10130000EBEC26F041EC24F00A0EACEC23F0170FC6
:10131000A6EC21F0090FB0EC29F0070EACEC23F09D
:101320000C0FA6EC21F00D0FE3EC26F049EC38F0A1
:1013300025EC27F0010EACEC23F0210FA6EC21F0F8
:101340000C0F9BEC22F0010EDB6A38EC26F0080E45
:101350008AEC25F011E299EC24F00F015CEC27F007
:10136000EF50200806E199EC24F05CEC27F0300EF9
:10137000EF6E010EDB2AE9D7D950230FA6EC21F03E
:10138000140FECEC29F0D950060FE6EC22F042EFF6
:1013900021F05BEC21F05E0EE126D950010F7BECD1
:1013A00025F0500EEE6E4C0EEE6E530E8BEC22F0CE
:1013B000EE6E51EC28F0120F7BEC25F04F0EEE6E26
:1013C000500EEE6E4E0E8BEC22F0EE6E08EC24F01A
:1013D0005B0EEE6E6D0EEE6E730EC0EC25F0280FF8
:1013E0005BEC2AF0250EEE6E5D0E5EEC25F0D9501A
:1013F0002D0F5FEC26F02E0EEE6E2D0EEE6EEE6EC5
:10140000EE6A3A0EDB6A4B0EDB6AD9505C0FEBECEE
:1014100026F0B60EEE6E010EED6ED950010FA6EC61
:1014200021F03A0F21EC28F0120FA6EC21F04B0F1F
:101430004CEC21F05FEC24F0EE50ED1007E05FEC97
:1014400024F01BEC28F0EE50ED1009E1D9502D0FDF
:10145000A6EC21F0410F21EC28F02D0F11D0FDEC6E
:1014600029F0F1EC27F0340FA6EC21F0410F4CEC01
:1014700021F0FDEC29F01BEC28F0F1EC27F0340F03
:10148000A6EC21F0520F21EC28F0230FA6EC21F05E
:10149000460F21EC28F0280FA6EC21F0570F4CEC5A
:1014A00021F0DF6A020EDF5C0AE2DF288AEC28F016
:1014B0003A0F39EC23F08FEC28F0DF2AF3D742EF14
:1014C00021F05BEC21F0310EE126D9501D0FEBEC41
:1014D00026F0680E51EC28F01F0FEBEC26F06D0E95
:1014E000E7EC25F0730E08EC24F04C0E51EC28F0DC
:1014F000250FC4EC25F0EE6A270EDB6A030EF36EAF
:10150000280EF3CFDBFF060EF36E290EF3CFDBFFC1
:10151000010EDB6A0101755102E0750505E1D95044
:101520001B0F34EC25F00AD0020E755D03E0030EAC
:10153000755D05E1D9501B0F39EC25F0ED6E74ECAB
:1015400026F02D0EEECFDBFF2E0EEECFDBFF2F0EA3
:10155000EECFDBFF300EEECFDBFFFEEC24F074ECC1
:1015600026F044EC29F0B5EC23F0190E1CC0DBFF8B
:101570001A0E1DC0DBFFD7EC27F00FEC29F0246A10
:1015800027EC3AF02A0EF6EC24F00FEC29F0FDECF3
:1015900021F0600E216EEA0E226E236A246A27EC87
:1015A0003AF02B0EF6EC24F0600E216EEA0E226E5D
:1015B000236AFDEC21F050EC29F02C0E1CC0DBFF5F
:1015C0003EEC25F02A0E9CEC27F0010F21EC28F0D0
:1015D0001D0FA6EC21F0030F4CEC21F03EEC25F0A2
:1015E0002B0E9CEC27F0040F21EC28F01F0FA6EC2B
:1015F00021F0060F4CEC21F03EEC25F02C0E9CEC7B
:1016000027F0070F21EC28F0210FA6EC21F0090F9D
:1016100021EC28F0250FA6EC21F00A0F4CEC21F06C
:10162000DBEC26F0120FE3EC26F0190EDBCFE6FF21
:101630001A0ECEEC27F0130FA6EC21F00B0F21ECC5
:1016400028F0230FA6EC21F0100F4CEC21F0DF6AFC
:10165000DF50006E016A030E8AEC25F010E283EC85
:1016600025F00F015CEC27F0EF50200806E183EC39
:1016700025F05CEC27F0300EEF6EDF2AE9D737EC6F
:1016800027F0D950010FE6EC22F042EF21F0C3EC35
:1016900028F00101765D03E1060E775D57E0890EC3
:1016A000DE6E010EDD6E020E006E0001F92BF951A7
:1016B000D880005402E3FA71F96BD8EC22F0EA0EFC
:1016C000EE1807E1030EED1804E1FA0517E1010138
:1016D00021D0D8EC22F0E90EEE1808E1030EED1847
:1016E00005E1FA050BE10101030E2FD0D8EC22F041
:1016F000E80EEE1806E1030EED1803E10101BD6BE3
:1017000025D0D8EC22F019EC23F0010193518AEC9A
:1017100025F002E3010E19D0D8EC22F019EC23F0E9
:1017200094518AEC25F010E3D8EC22F0EECF02F0D1
:10173000EFCF03F09351046E056A0450025C05502C
:10174000035802E2020E01D0030EBD6F42EF21F0FA
:101750005BEC21F0130EE1267EEC37F0120EDB6A13
:10176000DF6A39EC18F0000905E1010EF36E120E84
:10177000F3CFDBFF100EE66EE66AAC0EE66E6D0E82
:10178000A3EC24F0020EE66EF2EC21F0B4EC26F0AD
:10179000E66E23EC23F0120EDB5005E0E66ADFCFA5
:1017A000E6FFC4EC23F0DF50006E016A0150000A2E
:1017B000E8AE02D0013405D0C80ED8800054000E27
:1017C000015419E3DF50FE0BE842010B14E197ECE2
:1017D00025F0010FE3EC26F0DF50FE0BE842E66E49
:1017E000100E02EC24F0B4EC26F0E66E23EC23F0AD
:1017F000140EF1EC23F0DF2AFF0EDF5CCCE142EFA8
:1018000021F05BEC21F00A0EE12612EC25F0250E0A
:101810005EEC25F07EEF29F05BEC21F0090E7BEC0D
:1018200026F06B0EEE6E6D0E5EEC25F064EC26F08D
:10183000FE0EF0EC29F0D9CFE6FFC8EC25F0FD0E46
:10184000DBCFE6FFDAEC23F0040EE76EFC0EDBCF15
:1018500000F0FD0EDBCF01F05FEC27F0E7EC26F0A7
:1018600042EF21F058EC29F012EC25F04C0EEE6E10
:10187000EE6A7EEF29F05BEC21F0080E7BEC26F09F
:1018800072EC29F01DEC2AF09BC1E6FF65EC22F01A
:10189000D950010FE66E49EC22F0DAEC23F0020E8B
:1018A0005FEC2AF0F6EC21F0EF50200804E1F6ECB2
:1018B00021F0300EEF6E1DEC2AF09CC1E6FF65ECC6
:1018C00022F0ACEC29F0030E60EC21F0DAEC23F00E
:1018D000050E5FEC2AF01DEC2AF09DC1E6FF65ECD9
:1018E00022F0ACEC29F0060E5FEC2AF0080EE76E51
:1018F000F6EC21F07BEC24F0200EEF6E42EF21F0AD
:101900005BEC21F0220EE12601017851490A43E007
:10191000010A41E00F0A19E0010A3DE1C3EC26F09B
:101920007951EE5C7A51EE587B51EE587C51EE586D
:1019300032E2010EC86F7DC1D3F17EC1D4F17FC107
:10194000D5F180C1D6F1470E25D0C9C100F0CAC17A
:1019500001F0026A036AC3EC26F00CEC27F0005099
:10196000795D01507A5902507B5903507C5913E339
:10197000C86BD30EE96E010EEA6EEE507D5DD36F3B
:10198000EE507E59D46FEE507F59D56FEE5080598E
:10199000D66F480E786F5B0EDF6EFF0EC91909E136
:1019A000CA5107E10E0EE66EE66AF30EE66E6B0EA6
:1019B0000CD0FB0EC9190BE1030ECA1908E10E0E7B
:1019C000E66EE66A040EE66E6C0EA3EC24F05D0E85
:1019D000F36E0F0EF3CFDBFF100EDB6A01017851BF
:1019E000490A34E0010A2EE00F0A06E0010A43E149
:1019F000F10EE66E6C0E2DD0E00EE66E6C0EE66E0D
:101A0000D950110F87EC21F0C3EC26F0EE50010104
:101A1000795D006EEE507A59016EEE507B59026E80
:101A2000EE507C59036E00C0E6FF01C0E6FF02C025
:101A3000E6FFE66ED950140FE3EC26F0A8D825ECAB
:101A400027F00CD0020EE66E6D0E03D0130EE66E7C
:101A50006D0EE66ED950110F87EC21F0CFC1E6FF75
:101A6000D0C1E6FFD1C1E6FFD2C1E6FF08EC25F008
:101A700014D825EC27F0110EE66EE66A54EC29F036
:101A800069EC21F0110EACEC23F0110FE3EC26F021
:101A9000110E1DEC28F042EF21F05BEC21F00C0E52
:101AA000E12612EC25F072EC29F0090EDB6A030E38
:101AB000F36E0A0EDFEC26F016EC25F09F0ED880B0
:101AC000EE54860EEE54010EEE54000EEE5407E274
:101AD000630EC8EC26F0630E59EC25F025D0AAEC75
:101AE00024F050EC29F0050EF6EC24F0EAEC23F09B
:101AF00003EC27F025EC28F016EC25F04FEC27F04E
:101B0000F90E00C0DBFFFA0E01C0DBFFFB0E02C0C6
:101B1000DBFFFC0E03C0DBFFAAEC24F00A0E8EEC08
:101B200023F0060E1CC0DBFF1DEC2AF0050EF0ECC6
:101B300029F0020E31EC28F0070FE3EC26F0020E3C
:101B40001DEC28F01DEC2AF0060EF0EC29F0020E38
:101B5000E1EC29F0030E1DEC28F00B0EDB6A38ECEB
:101B600026F0020E8AEC25F010E2D950090F006E23
:101B70000B0E02EC2AF006E1D950090F006E0B0E95
:101B800008EC2AF00B0EDB2AEAD742EF21F05BECDF
:101B900021F00F0EE126B9EC23F072EC29F0020ED1
:101BA000F36E0D0EDFEC26F016EC25F0F30ED88068
:101BB000EE54090EEE54000EEE54000EEE540EE2FA
:101BC000F30EF36EF90EF3CFDBFF090EF36EFA0E90
:101BD000F3CFDBFFFB0EDB6AFC0EDB6AD950070F8D
:101BE000A6EC21F016EC25F032EC24F0FBEC26F00C
:101BF000090EDBCFE6FF0A0EDBCFE6FF81EC22F019
:101C0000030E31EC28F00B0FE3EC26F0030E1DEC75
:101C100028F0010EACEC23F0040FE3EC26F0040EE8
:101C20001DEC28F00E0EDB6A38EC26F0010E8AEC73
:101C300025F010E2D9500D0F006E0E0E02EC2AF0C6
:101C400006E1D9500D0F006E0E0E08EC2AF00E0EB4
:101C5000DB2AEAD742EF21F08AEC27F0340E0101AB
:101C6000785D06E0350E785D03E0360E785D0CE1B8
:101C7000340E785D02E1090E14D0350E785D02E174
:101C80000C0E0FD00F0E0DD00D0E785D09E00E0E6C
:101C9000785D06E00F0E785D03E0100E785D0BE1D5
:101CA0000F0EDF6E020EE66EDFCFE6FF5DEC29F071
:101CB000010EE66E01D0E66ACAEC37F0E55288EF15
:101CC00022F0C3EC28F0010EDE6EDD6A01016C0526
:101CD00008E1F60EDB5001E17ED0F60EDB50DE6E41
:101CE000DD6AD7EC26F034E162EC29F0FA0EDB5025
:101CF00000180AE1FB0EDB50011806E1F70EDB507D
:101D00001AE016EC29F019D0DECF02F0DDCF03F097
:101D10009FEC21F00250EE24006E0350EE20016E85
:101D2000FA0EDBCF04F0FB0EDBCF05F00050045CB5
:101D30000150055805E21DEC29F0DBCFEDFF08D07E
:101D400063EC25F09FEC21F00050EE260150ED22CF
:101D5000FE0EDB5004083FE162EC29F0F80EDB5088
:101D600000180AE1F90EDB50011806E1F70EDB500E
:101D700025E01DEC29F024D062EC29F0DECF02F042
:101D8000DDCF03F00250005C0350015817E3DECFB3
:101D900006F0DDCF07F09FEC21F00650EE5C046EFC
:101DA0000750EE58056EF80EDBCF08F0F90EDBCFCA
:101DB00009F00850045C0950055805E216EC29F0BA
:101DC000DBCFEDFF08D063EC25F09FEC21F0005055
:101DD000EE5E0150ED5A42EF21F05BEC21F0140E63
:101DE000E126D950110FEBEC25F0050E0101752508
:101DF000E76E130EE7CFDBFFDBCFE6FF110EDBCF85
:101E0000E9FF120EDBCFEAFFEF50E552E75C110D60
:101E1000F350026E036A110EDBCFE9FF120E28ECBD
:101E200024F032EC25F037EC27F0100EE66ED9CF17
:101E3000E6FF23EC23F042EF21F058EC29F0D950D3
:101E4000010F5BEC2AF0590EC0EC25F0050F5BEC9E
:101E50002AF04E0EEE6E5D0EEE6EEE6A0D0E010174
:101E6000785D03E1A2C1DFFF11D00E0E785D03E1C2
:101E7000A3C1DFFF0BD00F0E785D03E1A4C1DFFF2C
:101E800005D0100E785D02E1A5C1DFFFDF0403E19C
:101E9000D950010F02D0D950050F27EF2AF05BEC83
:101EA00021F00C0E6FEC26F0CB0EEE6ED90E51EC3D
:101EB00028F0090FEBEC26F0D60EEE6ED90EEE6E82
:101EC000EE6A0101BA5102E0BA052BE1C0EC27F03D
:101ED000EFCFDFFFBA5105E1020EACEC23F0060FA5
:101EE00006D0BA051EE1020EACEC23F0090FE66E37
:101EF00049EC22F069EC21F0040E60EC21F0DFCF18
:101F0000E6FF070E02EC24F0E66AACEC29F0DFCF26
:101F1000E6FF65EC22F0030EE1EC29F00C0E1DEC5F
:101F200028F042EF21F0CCEC28F012E10101BD05D0
:101F300002E1808212D0020EBD5D02E1808203D0F8
:101F4000030EBD5D02E1808408D0BD5106E103D0DF
:101F5000FE0EDB5002E18092809482EF27F08AEC43
:101F600027F0DF6A8050100B100A01E0010EE82410
:101F7000DF128050200B200A01E0010EDF12DF503B
:101F800088EF22F0E66A49D8E55268EC25F0650E44
:101F9000E66E86EC3AF0E5527E0EE66E15EC3BF00E
:101FA000E552FA0ECB6E7D0EE66E69EC3AF0E55224
:101FB000E66ADAEC34F0E552840EAFEC26F0B19C20
:101FC000850EE66E3EEC3BF0E552030E74EC22F01B
:101FD000040EBEEC29F0100E74EC22F0110E74EC1D
:101FE00022F0120E74EC22F0090E74EC22F00A0EAC
:101FF00074EC22F00B0E74EC22F00D0E74EC22F057
:102000002DEC2AF00C0E74EC22F00E0E74EC22F083
:102010000F0E74EC22F066EF24F0CCEC28F002E115
:10202000D08E04D0FE0EDB5001E1D09E82EF27F06F
:102030005BEC21F0110EE12624EC29F032EC25F0C6
:10204000100EDB6AFBEC26F08FEC28F042EF21F05B
:102050008AEC27F0020E0101765D03E1060E775D42
:102060002CE0BA5117E1DF6A8250200B02E1010E29
:1020700001D0000E000919E0190EF1EC23F0825096
:10208000200B02E1010E01D0000E00090EE0010E4E
:10209000DF6E0BD0010EDF6E8250200B02E1010ECD
:1020A00001D0010E000901E0DF6ADF500101BA5DD5
:1020B00004E0DFCFBAF1C9EC23F088EF22F08AEC1C
:1020C00027F0DF6A8150010B02E0010E01D0000E03
:1020D00000090DE0190EF1EC23F08150010B02E034
:1020E000010E01D0000E000902E0010EDF6EDF508C
:1020F00088EF22F01200E66ADAEC34F0E552100EB6
:102100008EEC27F0D8EC34F068EC25F0F292B6ECC7
:102110003BF07EEC37F082909268936894681200EE
:102120008EEC25F04AEC26F01DEC25F0100E7EEC2E
:1021300027F080960101010E686F576B586B766B24
:1021400082961200BEEC28F0020EDB6AE66ACAEC48
:1021500033F0E552DF6E190EF1EC23F0E66ACAECBB
:1021600033F0E55203EC25F0DF50006E016AFF0EFC
:10217000001801E1015009E0010EDB50026E036A14
:10218000FF0E021804E1035002E1000E6ED0010EB2
:10219000DB04006EDF50D880005405E3010EDB281D
:1021A000D880DF5402E2FF0E60D0100E006EDF50C8
:1021B000005C05E22E0EDF5C02E2010E4ED0440E02
:1021C000006EDF50005C11E2DF50016E026A0250C7
:1021D000000AE8AE02D0D89004D08F0E015C000E49
:1021E000025803E2020EF36E3AD08D0E006E016AC1
:1021F000DF50000101AF02D0D89003D0005D000E87
:10220000015910E2DF50026E036A0350000AE8AE83
:1022100002D0D89004D0AB0E025C000E035802E24C
:10222000030E1BD0BA0E006E016ADF5001AF02D060
:10223000D89003D0005D000E015914E2DF50026E09
:10224000036A0350000AE8AE02D0D89004D0D80E3A
:10225000025C000E035806E2040EF36E020EF3CF8A
:10226000DBFF02D0020EDB68DB5042EF21F08AEC8C
:1022700027F0DF6801017651030A12E0010A0CE041
:10228000030A06E0010A12E1A1EC29F012D80BD0F2
:10229000A1EC29F048D807D0A1EC29F07AD803D0D6
:1022A000A1EC29F0D0D9E552E552E552DF5088EF94
:1022B00022F05BEC21F0040EE126D950020FEBEC8A
:1022C00025F0FE0EDB0413E10101010E766F776B42
:1022D0009FEC21F0010EEF6E19EC25F0F1EC25F0EA
:1022E000D4EC27F0DEEC28F0D4EC27F01AD0D7ECB1
:1022F00026F004E0FE0EDB50040813E1050E010198
:1023000075253CEC27F063EC25F0050E005E000E11
:10231000015A00C075F19FEC21F0EF6A0101070E30
:102320006E6F42EF21F0CCEC28F00DE10101772B2C
:102330000A0E006E7751005C01E2776B9FEC21F092
:10234000010EEF6E24D0FE0EDB50020820E10A0ED3
:102350000101775D03E183EC28F019D0020E766F5E
:1023600078699FEC21F0020EEF6E060E775D0FE1AB
:10237000070EE66EE66ABA0EE66E010EE66EC10E56
:10238000E66E010ED4EC27F00101020EBD6F82EF64
:1023900027F05BEC21F0040E8FEC24F06DEC24F0C0
:1023A000FE0EDB043AE1770503E0020E775D05E1FE
:1023B00019EC25F0F1EC25F019D0050E775D03E15D
:1023C000DEEC28F013D0060E775D0BE1070EE66E0B
:1023D000E66AC10EE66E010EE66EBA0EE66E010EFC
:1023E00005D0040E775D05E127EC25F0E66E69EC7B
:1023F00021F0460E006E01017851D880005406E3AA
:102400007851490803E383EC28F01BD1010E766F65
:1024100078699FEC21F0010E13D1FE0EDB5002080B
:102420001FE1330E54EC25F003E3785136080BE23C
:10243000640E016E7851D880015403E37851660828
:1024400002E278C16DF1020EDBCFE6FF030EDBCFB7
:10245000E6FF9BEC1DF0E552E5520101786FEDD0EF
:10246000D7EC26F005E0FE0EDB50040801E0E9D0D1
:1024700077513FE1785101E1DBD0780501E1D8D017
:10248000340E785D0EE19B51DE6EDD6AE66AE66A27
:10249000000EE66EE66A630E6DEC21F0DFCF9BF175
:1024A000CCD0350E785D09E19C510DEC24F00C0E7A
:1024B0006DEC21F0DFCF9CF1C0D0360E785D09E1E4
:1024C0009D510DEC24F01F0E6DEC21F0DFCF9DF13E
:1024D000B4D0330E785D01E0B0D00A0EE66EE66A45
:1024E000000EE66EE66AE668E668990EE66E010E94
:1024F0000ED0770510E10A0EE66EE66A76EC29F05A
:102500002F0EE66E750EE66E950EE66E010EE66E09
:1025100099EC28F092D0020E775D19E1030E785DF8
:1025200009E197510DEC24F0FA0E6DEC21F0DFCFAC
:1025300097F183D0040E785D01E07FD098510DECC7
:1025400024F0FA0E6DEC21F0DFCF98F176D0030E77
:10255000775D6EE0040E775D07E10B0E785D68E055
:102560000C0E785D6AE164D0050E775D37E10D0EE3
:10257000785D02E1A2510ED00E0E785D02E1A3510A
:1025800009D00F0E785D02E1A45104D0100E785DE1
:1025900003E1A551DE6EDD6AE66A010EE66E000E0D
:1025A000E66EE66A010E6DEC21F00D0E0101785D1C
:1025B00003E1DFCFA2F141D00E0E785D03E1DFCF62
:1025C000A3F13BD00F0E785D03E1DFCFA4F135D04E
:1025D000100E785D32E1DFCFA5F12FD0060E775DCA
:1025E0001EE1C0EC27F0EF50DE6EDD6AD7EC26F07E
:1025F00002E1040E01D0030EF36EFE0EF3CFDBFFFB
:1026000076EC29F0E66EE66A640E6DEC21F00101CD
:10261000C0EC27F0DFCFEFFFC9EC23F00ED0070EA0
:10262000775D0BE0080E775D08E0090E775D05E148
:1026300078513CEC27F0DFCF78F19FEC21F0020ECF
:10264000EF6E42EF21F0CCEC28F003E1010183ECC6
:1026500028F082EF27F05BEC21F0130EE126240E28
:10266000E66E6D0EE66ED950020F87EC21F0870EF4
:10267000E66ECAEC33F0E552DF6EE66AD9500C0F15
:10268000E3EC26F0DFCFE6FF65EC22F097EC25F0D7
:10269000020FE6EC22F042EF21F05BEC21F0080E95
:1026A0000CEC25F072EC29F0FB0EDB50020801E285
:1026B00077D0640EF9EC25F0020E1FC0DBFFDB5073
:1026C000640D9DEC25F00A0EF9EC25F0030E1FC0F9
:1026D000DBFFDB500A0D9DEC25F0DB50E76E040EAE
:1026E000E7CFDBFF070EDB6A030E66EC29F00DE295
:1026F00048EC28F0070EDB50A6EC22F0F8EC23F0B3
:1027000083EC2AF0070EDB2AEFD7FB0EDB5012E03A
:10271000FB0EA6EC25F0020E046EFB0EE4EC28F096
:10272000030E096EFB0EF4EC22F0020E046EFB0E9B
:1027300033EC2AF0FB0EDB500FE1070EDB6A020ED2
:1027400066EC29F01CE2D950F8EC23F0B3EC29F048
:1027500016E10FEC2AF0F3D7070EDB6A010E006ECC
:10276000FB0EDB04005C66EC29F009E2D950F8ECC2
:1027700023F0B3EC29F003E10FEC2AF0EFD7FB0EC6
:10278000DB5002E0060E01D0050EDB6AD950020FC5
:10279000E66EC8EC25F0FD0EDBCFE6FFE7EC26F099
:1027A00042EF21F05BEC21F00B0E0CEC25F072EC0B
:1027B00029F0FA0EDB50040801E2ADD0100E006ED5
:1027C000270E016ECCEC22F0020E1EC0DBFF38ECAF
:1027D00026F0100E0102F3CF01F0270E0002F35095
:1027E0000126100E0002F450012677EC23F0E80ECB
:1027F000006E030E016ECCEC22F0030E1EC0DBFF58
:1028000038EC26F0E80E0102F3CF01F0030E0002CF
:10281000F3500126E80E0002F450012677EC23F075
:10282000640E006E016ACCEC22F0040E1EC0DBFFC9
:10283000DB50640DF4CF01F077EC23F00A0E006E4C
:10284000016ACCEC22F0050E1EC0DBFFDB500A0D46
:1028500016EC28F077EC23F0FD0EDB50E76E060E49
:10286000E7CFDBFF090EDB6A050E6AEC29F00DE20B
:1028700048EC28F0090EDB50A6EC22F0FDEC23F02A
:1028800083EC2AF0090EDB2AEFD7FA0EDB5012E0B8
:10289000FA0EA6EC25F0040E046EFA0EE4EC28F015
:1028A000050E096EFA0EF4EC22F0040E046EFA0E18
:1028B00033EC2AF0FA0EDB500FE1090EDB6A040E4E
:1028C0006AEC29F01CE2D950FDEC23F0B3EC29F0BE
:1028D00016E116EC2AF0F3D7090EDB6A030E006E40
:1028E000FA0EDB04005C6AEC29F009E2D950FDEC39
:1028F00023F0B3EC29F003E116EC2AF0EFD7FA0E3F
:10290000DB5002E0080E01D0070EDB6AD950020F3F
:10291000E66E3DEC23F042EF21F05BEC21F00E0E71
:10292000E126FB0E3CEC28F000EC26F027EC3AF018
:10293000010E79EC22F000EC26F03CEC21F008ECE2
:1029400026F027EC3AF0020E79EC22F008EC26F0A3
:102950003CEC21F010EC26F027EC3AF0030E79EC79
:1029600022F010EC26F03CEC21F018EC26F027ECDD
:102970003AF0040E79EC22F018EC26F03CEC21F051
:10298000B5EC23F0050E79EC22F0ECEC28F03CECF1
:1029900021F0ABEC25F0060E79EC22F0C7EC27F025
:1029A0003CEC21F050EC29F0070E79EC22F0EAEC37
:1029B00023F03CEC21F0640E8EEC23F0080E79EC51
:1029C00022F0640ED1EC28F03CEC21F00A0E8EECE3
:1029D00023F0090E79EC22F00A0ED1EC28F0EFEC8E
:1029E00026F015EC27F0DB50E76E0A0EE7CFDBFF91
:1029F0000C0EDB6A0A0EF36E0C0EA1EC22F00FE255
:102A0000D950010F72EC2AF00C0EDB50A6EC22F02C
:102A10004AEC25F083EC2AF00C0EDB2AEBD70C0EE7
:102A2000DB6A090EF36E0C0EA1EC22F00EE2D95017
:102A30004AEC25F0B3EC29F008E1D9504AEC25F036
:102A400094EC28F00C0EDB2AECD70A0EE1EC29F00E
:102A5000F90EDBCFE6FFFA0EDBCFE6FF69EC21F0E3
:102A600042EF21F05BEC21F01F0EE126100E7DC13C
:102A7000DBFF110E7EC1DBFF120E7FC1DBFF130EE9
:102A800080C1DBFF140E79C1DBFF150E7AC1DBFFBD
:102A9000160E7BC1DBFF170E7CC1DBFF180E91C148
:102AA000DBFF190E92C1DBFF1A0E99C1DBFF1B0E73
:102AB0009AC1DBFF1C0E9DC1DBFF01019B39F00BAE
:102AC0009C11E76E1D0EE7CFDBFFE66A6DEC25F08B
:102AD000DF5006E0D30E006E0E0EDF24005C02E233
:102AE000010E02D00E0EDF24DF6E1E0EDB6A100E0A
:102AF000DBCF02F0110EDBCF03F0120EDBCF04F0C0
:102B0000130E2BEC29F0F8EC26F0DEEC22F0100F7F
:102B100050EC21F0080EB1EC21F0FDE199EC29F028
:102B200029EC23F0100F50EC21F0100EB1EC21F045
:102B3000FDE199EC29F031EC23F0100F50EC21F07D
:102B4000180EB1EC21F0FDE199EC29F002C0EFFF85
:102B5000140EDBCF02F0150EDBCF03F0160EDBCF29
:102B600004F0170E2BEC29F046EC21F0DEEC22F0FD
:102B7000140F50EC21F0080EB1EC21F0FDE199ECBE
:102B800029F029EC23F0140F50EC21F0100EB1ECD9
:102B900021F0FDE199EC29F031EC23F0140F50EC19
:102BA00021F0180EB1EC21F0FDE199EC29F002C002
:102BB000EFFFFF0EE76E80EC26F0E750021679EC8F
:102BC00027F080EC26F0C6EC29F0FF0EE76E87ECCC
:102BD00026F0E750021679EC27F087EC26F0C6ECD9
:102BE00029F063EC2AF01C0EDBCFEFFF63EC2AF038
:102BF0001D0EDBCFEFFF010EDB6A0E0EC8EC28F0D6
:102C000005E2D950020FCEEC29F0F7D7DFCFE6FF6F
:102C1000E66AC4EC23F042EF21F05BEC21F02E0ECB
:102C2000E126D30EF36E240EF3CFDBFFE30EF36E3B
:102C3000250EDFEC26F0260F4BEC29F0280FE5ECF3
:102C400023F0ED6ED9502A0F34EC25F0ED6ED950FB
:102C50002C0F39EC25F0ED6E020EDB6AF36EDBCF44
:102C6000F4FFE850F45C01E3DAD0D950260FD6EC3B
:102C700028F0130EEECFDBFF71EC25F0D950260FB4
:102C800094EC21F0170EEECFDBFF180EEECFDBFF3A
:102C9000190EEECFDBFF1A0EEECFDBFFD9502A0F55
:102CA00094EC21F01B0EEECFDBFF1C0EEECFDBFF12
:102CB0001D0EEECFDBFF1E0EEECFDBFFD9502A0F2D
:102CC000D6EC28F01F0EEECFDBFF200EEECFDBFFA1
:102CD000210EEECFDBFF220EEECFDBFFD950240F0B
:102CE000006E39EC2AF0230EDB6A130EDBCF02F004
:102CF000140E150E160E64EC27F0130F50EC21F095
:102D0000080EB1EC21F0FDE179EC2AF0130F50EC44
:102D100021F0100EB1EC21F0FDE17CEC2AF0130F54
:102D200050EC21F0180EB1EC21F0FDE17FEC2AF01F
:102D3000170EDBCF02F0180E190E1A0E64EC27F0F6
:102D4000170F50EC21F0080EB1EC21F0FDE179EC09
:102D50002AF0170F50EC21F0100EB1EC21F0FDE13C
:102D60007CEC2AF0170F50EC21F0180EB1EC21F09A
:102D7000FDE17FEC2AF01B0EDBCF02F01C0E1D0ED6
:102D80001E0E64EC27F01B0F50EC21F0080EB1EC86
:102D900021F0FDE179EC2AF01B0F50EC21F0100E30
:102DA000B1EC21F0FDE17CEC2AF01B0F50EC21F09E
:102DB000180EB1EC21F0FDE17FEC2AF01F0EDBCF05
:102DC00002F0200E210E220E64EC27F01F0F50ECB3
:102DD00021F0080EB1EC21F0FDE179EC2AF01F0F93
:102DE00050EC21F0100EB1EC21F0FDE17CEC2AF06A
:102DF0001F0F50EC21F0180EB1EC21F0FDE17FEC3B
:102E00002AF0010EDB6A100EC8EC28F005E2D9505A
:102E1000030FCEEC29F0F7D7020EDB2A1FD742EFC3
:102E200021F05BEC21F02D0EE126D30EF36E230E84
:102E3000F3CFDBFFE30EF36E240EDFEC26F0250F5D
:102E40004BEC29F0270FE5EC23F0ED6ED950290F5C
:102E500034EC25F0ED6ED9502B0F39EC25F0ED6EEA
:102E6000020EDB6AF36EDBCFF4FFE850F45C01E3A3
:102E7000FED0D950230F86EC27F039EC2AF0030E50
:102E800076EC2AF0130E00C0DBFF8EEC26F047EC48
:102E900023F003E035EC22F0FDE1CBEC21F0020E53
:102EA000AAEC21F0130F7CEC21F0CBEC21F047ECE5
:102EB00023F003E035EC22F0FDE1CBEC21F0DF283C
:102EC000E66E20EC2AF066EC28F047EC23F003E0F5
:102ED00035EC22F0FDE1CBEC21F0CEEC25F066ECF8
:102EE00028F0070E76EC2AF0170E00C0DBFF95ECF9
:102EF00026F053EC23F003E035EC22F0FDE1D8ECB2
:102F000021F0060EF9EC27F053EC23F003E035EC4A
:102F100022F0FDE1D8EC21F0050EF9EC27F053EC9E
:102F200023F003E035EC22F0FDE1D8EC21F0040EB3
:102F3000F9EC27F0080E76EC2AF01B0E00C0DBFF40
:102F40001C0EDB6A1D0EDB6A1E0EDB6A5FEC23F0D3
:102F500003E035EC22F0FDE13CEC22F0090E00EC40
:102F600028F05FEC23F003E035EC22F0FDE13CECCF
:102F700022F00A0E00EC28F05FEC23F003E035ECC1
:102F800022F0FDE13CEC22F00B0E00EC28F00F0EDD
:102F900076EC2AF01F0E00C0DBFF200EDB6A210E4C
:102FA000DB6A220EDB6A6BEC23F003E035EC22F0E7
:102FB000FDE1E5EC21F00E0E07EC28F06BEC23F0C0
:102FC00003E035EC22F0FDE1E5EC21F00D0E07EC1D
:102FD00028F06BEC23F003E035EC22F0FDE1E5ECAA
:102FE00021F00C0E07EC28F0D950250FD6EC28F074
:102FF000130EDBCFEEFF140EDBCFEEFF150EDBCF93
:10300000EEFF160EDBCFEEFFD950250F94EC21F02A
:10301000170EDBCFEEFF180EDBCFEEFF190EDBCF66
:10302000EEFF1A0EDBCFEEFFD950290F94EC21F002
:103030001B0EDBCFEEFF1C0EDBCFEEFF1D0EDBCF3A
:10304000EEFF1E0EDBCFEEFFD950290FD6EC28F095
:103050001F0EDBCFEEFF200EDBCFEEFF210EDBCF0E
:10306000EEFF220EDBCFEEFF020EDB2AFBD642EF95
:1030700021F08AEC27F0DF6AFE0EDF5C08E2CEEC7E
:1030800025F0FF0802E0010E03D0DF2AF5D7000E7D
:1030900088EF22F08AEC27F0DF6AE66ADF50DF2A49
:1030A00024EC2AF0FF0EDF5CF8E188EF22F08AECD6
:1030B00027F076EC29F0C4EC23F0DF6AD20EDF5C57
:1030C00006E2E66ADF2824EC2AF0DF2AF7D788EF49
:1030D00022F058EC29F0360EC8EC26F0310E59ECEF
:1030E00025F0300EB9EC26F0300EF36E080EF3CF5B
:1030F000DBFF8250100B02E0010E01D0000E000930
:1031000001E094D0DF6A020EDF5C13E2DF28E66E96
:10311000F2EC21F0DF50110D16EC28F0680E0026BD
:103120006D0EE6EC29F018EC10F0E552E552DF2ABE
:10313000EAD768EC25F00B0E8EEC27F066EC24F055
:10314000DF6A030EDF5C6DE20101726B040EDB6A65
:10315000030EDB6A020E725D3AE1DF6AD30EDF5CBA
:1031600015E2CEEC25F0E76E020EE7CFDBFFD2ECE6
:1031700025F0030EDBCFE7FF020EDB50E71A030E4C
:10318000E7CFDBFFACA2FED7DF2AE8D7DF6A040E69
:10319000DF5C17E2D950050FDDEC29F0EF50E2ECCF
:1031A00025F0D950050FDDEC29F0030EDBCFE7FF4A
:1031B000EF50E71A030EE7CFDBFFACA2FED7DF2A02
:1031C000E6D7030ED2EC25F0ACB20CD0FDD782507E
:1031D000100B02E0010E01D0000E0009BBE0010E51
:1031E000DDEC25F0040EDB041CE0010EDB6A1E0E94
:1031F000C8EC28F011E2060E0101725D04E1010E37
:10320000DDEC25F009D0150E725D06E00A0EF1EC3A
:1032100023F0010EDB2AEBD7040EDB0402E0DF2AE9
:1032200090D768EC25F00B0E7EEC27F042EF21F0F2
:10323000BEEC28F0E66A6DEC25F0DF5006E0D30E18
:10324000006E0D0EDF24005C07E2010ECDEC26F0CF
:10325000DE52510EDD6E39D00C0E75EC27F0E76EA4
:10326000020EE7CFDBFF0D0E75EC27F003EC25F027
:10327000020EDB5006E01F0E006E020EDB50005CFB
:1032800003E2010ECDEC26F0010EDB500F0B006EB9
:10329000010E005C07E30C0E016E010EDB500F0BFC
:1032A000015C06E2010EDB50F00B010903EC25F096
:1032B000630E006E010ED2EC26F0005C06E2010EF9
:1032C000DB500F0B500903EC25F0010ED2EC26F079
:1032D00001019B6F010EDB500F0B9C6F020EDBCFC9
:1032E0009DF142EF21F05BEC21F0040EE126F30E9C
:1032F000E66E6DEC25F0F40EE66E20EC2AF003ECA1
:1033000025F0DB50E66ED950020FEBEC26F0E552CB
:10331000E750EE6EED6A74EC24F000C001F0006A34
:103320006DEC24F0DF50E76E74EC24F0E7500012EF
:103330006DEC24F074EC24F0010E8AEC25F00CE323
:10334000020EDBCF02F0030EDBCF03F02F0ED8808E
:103350000254750E035406E2100ECDEC26F0270E33
:10336000BEEC26F0020EDBCF91F1030EDBCF92F123
:1033700042EF21F001019151E66EF30E24EC2AF0A8
:103380000101FF0E9215006E016AE850E66EF40E20
:1033900024EF2AF08AEC27F0F50EE66E6DEC25F0AE
:1033A000DFBE03D055EC28F016D0080EDF14E8403D
:1033B000E840E8401F0B01019E6F040EDF14E84057
:1033C000E8403F0B9F6F020EDF14E8407F0BA06FB9
:1033D000010EDF14A16F88EF22F08AEC27F0DF6A7C
:1033E0000101A15101E0DF80A05101E0DF829F5186
:1033F00001E0DF849E5101E0DF86DF8EDFCFE6FF54
:10340000F50E24EC2AF088EF22F05BEC21F00C0E94
:10341000E126750EDDEC25F0C80EC8EC26F04D0E49
:1034200059EC25F0730EB9EC26F043EC25F0FD0EB7
:10343000DBCF02F0FE0E3FEC2AF0040EDBCF22F0D1
:10344000050EDBCF23F0060EDBCF24F0070EDBCF1B
:1034500025F0F8EC30F01DC0DEFF1EC0DEFF1FC0FF
:10346000DEFF20C0DDFFDD52DD52DECF1DF0DECFFE
:103470001EF0DECF1FF0DDCF20F0DD52DD52C0ECBC
:1034800031F01EC000F01FC001F09CEC26F01EC001
:10349000EEFF01C0EDFFD9CFE9FFDACFEAFFA3ECE1
:1034A00026F0EFCF03F020EC26F0A1EC27F0F8ECAB
:1034B00030F05EEC32F092EC23F0216E270E226E9B
:1034C000236A246AEFEC26F027EC3AF0D4EC29F0DA
:1034D000020EE76E9CEC26F07BEC24F018C0EEFFA9
:1034E00001C0EDFF42EF21F001010651DFEC23F0B6
:1034F000070EE926010EEA22BECFEEFFBFCFEDFF99
:1035000012005BEC21F00B0EE12679C102F17AC1C9
:1035100003F17BC104F17CC105F10101065108E111
:1035200079C159F17AC15AF17BC15BF17CC15CF17F
:103530000651062BDFEC23F01B0EE926010EEA22D2
:10354000BECFEEFFBFCFEDFF0A0E006E0651D88052
:10355000005418E3280EE66EE66A070EE66E010ECA
:10356000E66E2F0EE66E010ED4EC27F059C15DF128
:103570005AC15EF15BC15FF15CC160F10101066B94
:10358000010E616F42EF21F05BEC21F0270EE12686
:103590008250080B01E0010EE66E7CEC33F0E55240
:1035A000010EDF6E090EDF5C43E2DAEC28F00EEC70
:1035B00028F0EECF02F0EFCF03F00050025C015094
:1035C000035834E26AEC22F0030EEECFDBFF040E68
:1035D000EDCFDBFF1EEC24F0010EEECFDBFF020E81
:1035E000EDCFDBFF0EEC28F019EC23F06AEC22F0B3
:1035F00000C0EEFF01C0EDFFF4EC28F019EC23F061
:103600001EEC24F000C0EEFF01C0EDFF0EEC28F030
:10361000030EDBCFEEFF040EDBCFEDFFF4EC28F062
:10362000010EDBCFEEFF020EDBCFEDFFDF2ABAD7B4
:103630000B0EDB6A0C0EDB6A0D0EDB6A0E0EDB6A0C
:10364000130EDB6A8EEC26F0170EDB6A95EC26F083
:10365000010EDF6E0A0EDF5C4DE2DAEC28F0026A42
:10366000036AB9EC23F00CEC27F0B7EC24F0DAECA9
:1036700028F0026A036AD950130F67EC2AF0CBECEA
:1036800021F01EEC24F019EC23F0026A036AD950F1
:10369000170F67EC2AF0D8EC21F0DAEC28F0710E65
:1036A000005C020E01580CE370EC28F0DBCF03F055
:1036B000710E005E020E015A000E025A035A16D015
:1036C0006AEC22F0EECF04F0EFCF05F0066A076A4D
:1036D000B9EC23F00450EE5C006E0550EE58016E1C
:1036E0000650EE58026E0750EE58036EB7EC24F009
:1036F000DF2AB0D745C108F046C109F00A6A0B6A53
:10370000B9EC23F00850EE5C046E0950EE58056EDB
:103710000A50EE58066E0B50EE58076E53C10CF06F
:1037200054C10DF00E6A0F6A0C50045C006E0D500F
:103730000558016E0E500658026E0F500758036E62
:103740000F0E00C0DBFF100E01C0DBFF110E02C028
:10375000DBFF120E03C0DBFFC4EC24F0070E8EEC7F
:1037600023F0D1EC24F0DEEC24F0090E8EEC23F0F3
:10377000130E1CC0DBFF140E1DC0DBFF150E1EC098
:10378000DBFF160E1FC0DBFF170EDBCF1CF0180E81
:10379000DBCF1DF0190EDBCF1EF01A0EDBCF1FF0B2
:1037A000090E8EEC23F0170E1CC0DBFF180E1DC097
:1037B000DBFF190E1EC0DBFF1A0E1FC0DBFF810EE0
:1037C000F36E1B0EF3CFDBFF0A0EF36E1C0EF3CF6E
:1037D000DBFF280EF36E1D0EF3CFDBFF7B0EF36EC7
:1037E0001E0EF3CFDBFF70EC28F007EC23F00B0E7E
:1037F0001CC0DBFF0C0E1DC0DBFF0D0E1EC0DBFF6F
:103800000E0E1FC0DBFF0F0EDBCF00F0100EDBCF64
:1038100001F0110EDBCF02F0120E07EC23F0D1EC19
:1038200024F0C4EC24F00A0ED1EC28F0C1EC39F0FD
:103830000F0E18C0DBFF100E19C0DBFF110E1AC0EF
:10384000DBFF120E1BC0DBFFB9EC23F001017D5141
:10385000EE24006E7E51EE20016E7F51EE20026E4E
:103860008051EE20036EE5EC21F0B9EC23F0855198
:10387000EE24006E8651EE20016E8751EE20026E1E
:103880008851EE20036E51EC26F0250E02C0DBFFBE
:10389000260E03C0DBFFFEEC24F0D9501F0F44ECD2
:1038A0002AF01CC089F11DC08AF1FEEC24F0D95029
:1038B000230F44EC2AF01CC08DF11DC08EF11F0EA9
:1038C000DBCF7DF1200EDBCF7EF1210EDBCF7FF150
:1038D000220EDBCF80F1230EDBCF85F1240EDBCF70
:1038E00086F1250EDBCF87F1260EDBCF88F1DEECEB
:1038F00024F0030ED8901C361D361E361F36E806FF
:10390000F9E1640E8EEC23F01CC0B6F11DC0B7F1D6
:10391000130EDBCF08F0140EDBCF09F0150EDBCF52
:103920000AF0160EDBCF0BF008C01CF009C01DF02A
:103930000AC01EF00BC01FF034EC2BF0AEEC25F0EB
:10394000170EDBCF10F0180EDBCF11F0190EDBCF06
:1039500012F01A0EDBCF13F0D950130FEBEC26F058
:10396000EE501026EE501122EE501222EE5013228D
:1039700010C01CF011C01DF012C01EF013C01FF0CB
:1039800034EC2BF01DC00CF01EC00DF01FC00EF06B
:1039900020C00FF014EC24F071EC2EF080EC23F03A
:1039A00020EC26F0F8EC30F0C0EC31F01EC0B8F19D
:1039B0001FC0B9F1070E79C1DBFF080E7AC1DBFF2A
:1039C000090E7BC1DBFF0A0E7CC1DBFF12EC25F088
:1039D00001015D51EE5C006E5E51EE58016E5F516B
:1039E000EE58026E6051EE58036E070E00C0DBFF0A
:1039F000080E01C0DBFF090E02C0DBFF0A0E03C088
:103A0000DBFF070EDBCF00F0080EDBCF01F0090E65
:103A1000DBCF02F00A0EDBCF03F0005001100210E2
:103A2000031025E1E90E8B6F030E8C6FE90E8F6F8B
:103A3000030E906FB9EC23F0AA51EE24AA6FAB519C
:103A4000EE20AB6FAC51EE20AC6FAD51EE20AD6F00
:103A5000B9EC23F0B251EE24B26FB351EE20B36F44
:103A6000B451EE20B46FB551EE20B56F5BD0070EA8
:103A7000DBCF04F0080EDBCF05F0090EDBCF06F03C
:103A80000A0EB7EC29F00C6A520E0D6E190E0E6E6E
:103A90008E0E0F6E1DC0E6FF1EC0E6FF1FC0E6FFC4
:103AA00020C0E6FF0CC0E6FF0DC0E6FF0EC0E6FF3B
:103AB000E66EFEEC24F0D9500F0FEBEC26F0C6ECCE
:103AC00021F0E552E7CF0FF0E552E7CF0EF0E552D7
:103AD000E7CF0DF0E552E7CF0CF0E552E7CF03F06A
:103AE000E552E7CF02F0E552E7CF01F0E552E7CF2C
:103AF00000F015EC22F01EC08BF11FC08CF11EC02F
:103B00008FF11FC090F10101E70ED8801E54030E03
:103B10001F5408E2E70E8B6F030E8C6FE70E8F6F5A
:103B2000030E906F8250080B01E0010EE66E7FECF1
:103B300033F0E552A7D38AEC27F078C1DFFF01010B
:103B4000775129E16D5127E1640E785D0EE118ECA3
:103B500019F089C199F18AC19AF10101A00502E128
:103B6000330E5FD09F0561E105D0330E785D04E12F
:103B70009F050FE1340E55D0340E785D02E1350E0D
:103B800050D0350E785D02E1360E4BD0360E785DA2
:103B90004CE1650E46D0020E775D05E1030E785DBF
:103BA00044E1040E3ED0050E775D13E10D0E785D05
:103BB00002E10E0EDF6E0E0E785D02E10F0E31D0C7
:103BC0000F0E785D32E1A30502E0A56B2ED0100E3A
:103BD00028D0040E775D29E10B0E785D03E00C0E12
:103BE000785D21E1C86B79C1CBF17AC1CCF17BC1A1
:103BF000CDF17CC1CEF1CF6BD06BD16BD26BD36BDF
:103C0000D46BD56BD66B0B0E785D03E1C969CA6BBB
:103C100007D00C0E785D04E1FB0EC96F030ECA6F6E
:103C2000460EDF6E02D0785136D07851DF5C02E06C
:103C3000DF5031D000EC27F0060804E1640E785D17
:103C400010E117D000EC27F0050804E1640E785D60
:103C500016E007D000EC27F0070807E1640E785D56
:103C600002E0640E13D0670E11D000EC27F00308B9
:103C700002E1650E0BD000EC27F0020802E1660EAF
:103C800005D000EC27F0040803E1670EDF6E02D0D8
:103C900078C1DFFFDF5088EF22F00DDB100EE12648
:103CA000006A016A0268036846EC24F0100ED8909E
:103CB0000332023201320032E806F9E100C0DEFFD1
:103CC00001C0DDFF00680168026A036A46EC24F067
:103CD0006DEC24F0B7EC25F063EC25F0B0EC22F0AD
:103CE000DBCF1CF0050EDBCF1DF0060EDBCF1EF088
:103CF000070EDBCF1FF0ABEC25F092EC23F01F0B8F
:103D000002E0B3DBFEE1E4EC27F0080EDBCF04F0C9
:103D1000090EDBCF05F00A0EDBCF06F00B0EDBCF72
:103D200007F0C7EC27F003EC27F0C1EC39F0D950CD
:103D3000040FEBEC26F04FEC27F0080E00C0DBFF81
:103D4000090E01C0DBFF0A0E02C0DBFF0B0E03C031
:103D5000DBFFB7EC25F074EC24F0B0EC22F0DBCF05
:103D600000F0050EDBCF01F0060EDBCF02F0070EF0
:103D7000DBCF03F092DB100E046ED950080FEBEC92
:103D800026F004501F0BA3EC26F0EECF03F002E068
:103D90006CDBFEE182DB0C0EDBCF00F00D0EDBCF27
:103DA00001F00E0EDBCF02F00F0EDBCF03F0EFECD5
:103DB00026F068D20101775120E1020ED8EC25F0FF
:103DC00001016D516EE19F5103E19B6B9C6B9D6BFB
:103DD000A05102E199699A6932EC15F00101A151F3
:103DE00009E0A05107E094D8F3CF91F1F4CF92F11C
:103DF000BAEC19F0010ED8EF25F0770506E195C170
:103E000091F196C192F1BAEF19F0020E775D05E1DA
:103E100097C193F198C194F11200030E775D1FE1F1
:103E2000050E6D5D02E1756B1200060E6D5D02E11F
:103E3000010E13D0070E6D5D02E1020E0ED0080ECA
:103E40006D5D02E1030E09D0090E6D5D02E1040E05
:103E500004D00A0E6D5D25E1050E756F1200050E8A
:103E6000775D0BE119EC25F0A20EE66E010EE66E11
:103E70004FEC25F02EDAEDEF19F0070E775D04E137
:103E80004AEC18F015EF03F0090E775D0AE1130E06
:103E90006D5D02E10DEF16F0140E6D5D02E111ECA7
:103EA00017F0120008DAA2DA0A0EEE26000EEE2251
:103EB000EE22EE2282EF27F0C3EC28F097DAEF50E3
:103EC0000DE0FD0EDBCFE9FFDB2AFE0EDBCFEAFFC4
:103ED00001E3DB2AEF50E2EC25F0F0D7FC0ED2EC48
:103EE00026F0300FDF6EFC0EDB500F0B300F03ECB3
:103EF00025F0DFCFE6FF64EC3BF0E552010ED2EC9B
:103F000025F00D0EE2EC25F00A0EE2EC25F0BAD118
:103F1000D2D9060EE12699C11EF09AC11FF086EC97
:103F20002AF0EEDB89C11EF08AC11FF086EC2AF070
:103F3000AEEC25F06CEC27F0A1EC27F071EC2EF044
:103F400081EC24F0DBCF04F0030EDBCF05F0040E90
:103F5000DBCF06F0050EDBCF07F091C11EF092C15A
:103F60001FF086EC2AF0ABEC28F014EC24F0F8EC0F
:103F700030F0C6DB226A236A246A7E0E256E7CEC52
:103F80002CF081EC24F0DBCF1DF0030EDBCF1EF014
:103F9000040EDBCF1FF0050EDBCF20F0C0EC31F0BC
:103FA0001EC0DEFF1FC0DDFF63EC25F000C0F3FF85
:103FB00001C0F4FF67D18AEC27F0F2AE03D0010E06
:103FC000DF6E01D0DF6A68EC25F0FE0EDB041EE137
:103FD00031EC29F0890EE66E010ED4EC27F028ECC6
:103FE00026F0790EE66E010ED4EC27F030EC26F0C8
:103FF000A60EE66E010ED4EC27F00101010E686FEB
:10400000026B036B046B056B066B19D0FE0EDB5065
:10401000020815E131EC29F08D0EE66E010ED4ECAC
:1040200027F028EC26F0810EE66E010ED4EC27F086
:1040300030EC26F0AE0EE66E010EE66E4AD9DF04D5
:1040400004E1E66A42EC34F0E55262D234D95C0E07
:10405000E126D950020FC4EC25F05B0EEE6E530E34
:10406000EE6E450EEE6E520EEE6E560EEE6E490E72
:10407000EE6E430EEE6E450EEE6E5F0EEE6E4D0E64
:10408000EE6E4F0EEE6E440EEE6E450EEE6E5D0E53
:104090005EEC25F0D950130FEBEC26F0CD0EEE6E52
:1040A000DD0EEE6EBA0EEE6EB30EEE6EBC0EEE6E62
:1040B000CF0EEE6EBC0EEE6EC00EEE6E200EEE6EED
:1040C000500EEE6E570EEE6E520EEE6E5F0EEE6EF0
:1040D0004F0EEE6E460EEE6E51EC28F0240FC4EC3F
:1040E00025F0EE6E530EEE6E500EEE6ECA0EEE6EB4
:1040F000DF0EEE6ED90EEE6EBD0E38EC29F05B0EC3
:10410000EE6E500EEE6E5D0EEE6E200EEE6EEE6EEC
:10411000EE6A020EF36E590EF3CFDBFF040EF36E60
:104120005A0EF3CFDBFF080EF36E5B0EF3CFDBFF0F
:10413000E66820EC2AF0080A09E00C0A05E0060A05
:1041400007E1580EDB6A09D0010E03D0020E01D040
:10415000010EF36E580EF3CFDBFF110EFDDA020FE6
:10416000F5D8360FB0EC29F0110EF6DA240FEED8A0
:10417000470FB0EC29F092EC29F0EBEC24F0350E6F
:10418000DB6A020EF36E350EDCD910E2350EDB2849
:104190008AEC28F0360F72EC2AF0350EDB507BECFF
:1041A00028F08FEC28F0350EDB2AEBD7A2EC10F0CC
:1041B0000009FCE1A2EC10F0DF6EDF500CE0FF0E16
:1041C000DF5C09E0010EDB5004E1DE52010EDD6E22
:1041D00006D0DF6A04D0DF5002E1010EDB6A020E76
:1041E000DF5C20E0030EDF5C03E0040EDF5C14E123
:1041F000030EDF5C0AE1580E38EC26F0020E8AEC62
:1042000025F00AE2580EDB2A07D0006A580EDB5070
:10421000005C02E2580EDB0692EC29F0DCDB49EC94
:104220002AF0C8D792EC29F0EF50E66EE668ACDAD7
:10423000110E92DA130F8AD8470FB0EC29F049EC2F
:104240002AF0FFD738D8050EE126E66AD9CFE6FF77
:10425000C8EC25F03AD9CAD8020EDBCFEFFF12D056
:104260008AEC27F0E6686DEC25F0FF0EDF5C02E1DA
:10427000040EDF6EDF504CD1EFEC26F015EC27F08A
:104280003CEF28F0D9CFE1FF82EF27F00024E96F5F
:10429000000EDA20EA6F1200E3EC26F0E7EF26F0DA
:1042A000EBEC26F0EE500216EE500316EE5004161C
:1042B000EE5005161200D9CFE6FFE1CFD9FF12006C
:1042C000E76EFD0EDBCF00F0FE0EDBCF01F05FEFFF
:1042D00027F01EEC38F025EF27F0E66E1DEC2AF0F3
:1042E00099EF28F0D950020F86EC27F01E0EDBCF95
:1042F000F3FFDB2AF3501200EBEC26F0EE50001235
:10430000EE500112EE500212EE5003121200E3ECD6
:1043100026F0FCEF28F0D950030F006E230EDBCF00
:10432000F3FFDB2AF3501200006E020EDB50020D89
:1043300005EC29F0EE50EFCFEAFFE96E1200FC0E1B
:10434000DBCFE9FFFD0EDBCFEAFF1200E3EC26F046
:10435000D950120076EC2AF0016A026A036AD95039
:104360001200D8900532043203320232E8061200FD
:104370001A0EDBCFE9FF1B0E6AEF2AF00F0D16ECC9
:1043800028F0920E00266A0E0CEF29F0AAEC27F016
:1043900084DC25EF27F0130E00C0DBFF140E01C0F4
:1043A000DBFF150E02C0DBFF160E03C0DBFF1200A1
:1043B000170E00C0DBFF180E01C0DBFF190E02C094
:1043C000DBFF1A0E03C0DBFF12001F0E00C0DBFF75
:1043D000200E01C0DBFF210E02C0DBFF220E03C056
:1043E000DBFF1200010EE66E5DEF29F0FD0EDBCF64
:1043F000E9FFFE0EDBCFEAFF1200246A03EC27F090
:1044000025EC28F02D0FEBEC26F04FEC27F02D0ECD
:1044100000C0DBFF2E0E01C0DBFF2F0E02C0DBFF52
:10442000300E03C0DBFFD7EF27F034EC2BF01DC0BC
:1044300010F01EC011F01FC012F020C013F06CEC81
:1044400027F00CC01DF00DC01EF00EC01FF00FC0F5
:1044500020F071EC2EF0ABEC28F06CEC27F0A1EC26
:1044600027F0F8EC30F0C0EF31F0D890003601368C
:1044700002360336E80612001B0E00C0DBFF1C0EDE
:1044800001C0DBFF1D0E02C0DBFF1E0E03C0DBFF01
:104490001200DACFE6FF24EF29F0C7EC27F0EFECAB
:1044A00026F027EC3AF01CC000F01DC001F01EC041
:1044B00002F01FC003F0D9500C0F67EC2AF0E4EFB4
:1044C00027F0B3EC27F04EEF2AF04DEC13F0E55255
:1044D0009DEF29F0EA6ADF34FE0BEA36E96E430EFF
:1044E000E926010EEA221200E66E8CEC34F0E55269
:1044F00012001CC0DBFFDBCF00F0016A026A036A16
:104500001200D2EC13F0F56E050EE15EF5501200CC
:10451000E55282EF27F038EC29F0EE6EEE6EEE6E8B
:10452000EE6EEE6E1200010EDBCFE9FF020EDBCF66
:10453000EAFFF4EF29F0E3EC26F0B6EC38F025EFD3
:1045400027F0DBCFF4FFF350F45C12000F0154ECC2
:104550002AF0E66EE4EC38F0E552E66ED95012002F
:10456000026A036AEFEC26F004C021F005C022F0D5
:1045700006C023F007C024F0C1EC39F0040E18C0C7
:10458000DBFF050E19C0DBFF060E1AC0DBFF070EAE
:104590001BC0DBFF040E1200FD0EDBCF1EF0FE0E73
:1045A000DBCF1FF000C023F001C024F0FFEF3AF092
:1045B000DECFE9FFDDCFEAFF1BEF28F06EEC29F03C
:1045C000026A0368046A056AD9501200E3EC26F017
:1045D0008FEF28F0DB04045C00010224006F000E62
:1045E000DA20016F6EEF2AF0DB04095C0724056F07
:1045F000000EDA20066F05C0E6FFE66E49EC38F0E3
:1046000025EC27F076EC29F0F6DB48EF28F03FECBC
:104610002AF01B0EDBCF22F01C0EDBCF23F01D0E89
:10462000DBCF24F01E0EDBCF25F0F8EC30F05EEF90
:1046300032F0EECF00F0EFCF01F01200E66E42EC68
:1046400034F0E5521200DACFE6FF89EC37F09DEF47
:1046500029F002C0EFFF026A036A0468056AD950B4
:10466000120002C0EFFF026A036A046A0568D950AB
:10467000120048EC29F07BEF28F0DACFE6FFFB0EC2
:10468000DBCFE6FFFC0EDBCFE6FFE7EF26F0130EF5
:10469000DBCF00F0140EDBCF01F0150EDBCF02F004
:1046A000160E4CEF28F0170EDBCF00F0180EDBCF04
:1046B00001F0190EDBCF02F01A0E4CEF28F01B0EA2
:1046C000DBCF00F01C0EDBCF01F01D0EDBCF02F0C4
:1046D0001E0E4CEF28F01F0EDBCF00F0200EDBCFBC
:1046E00001F0210EDBCF02F0220E4CEF28F0D95062
:1046F000FD0FF8EC29F0F350EE5E0150ED5A120078
:104700001DC000F01EC001F01FC002F020C003F069
:10471000120061DB790EEE6E010E1200D1EC28F072
:1047200027EF3AF0080E1CC0DBFF090E1DC0DBFFAF
:104730000A0E1EC0DBFF0B0E1FC0DBFF080EDBCF17
:1047400000F0090EDBCF01F00A0EDBCF02F00B0EFA
:10475000DBCF03F0100E1200E66EE66AD9501200AD
:10476000DBCFE9FF040E6AEF2AF0ECEC28F027EF2C
:104770003AF0D9500B0FEBEF26F0020EDBCFE9FF3A
:10478000030EDBCFEAFF1200E6EC34F0E552E5520F
:104790001200F6DBEF50E824320FC06FE850006ED5
:1047A000016AFA0ED8800056000E0156320E00241F
:1047B000BF6F12000CDBD950050FE3EF26F0E96E56
:1047C000EA6AD890E936EA36120005DB810EEE6E11
:1047D000010E1200E80E216E030E226E236A246A77
:1047E0001200E66EE66A82EC33F0E552E552120002
:1047F000020F8CDB070EDB501200020F87DB090E65
:10480000DB501200E66EDDEC05F0E5529DEF29F07D
:1048100051EC28F0230FEBEF26F0DE6EDD6A76EC2C
:1048200029F0E66EE66A120057DB04C01DF005C0F1
:104830001EF006C01FF007C020F01200EA6ADF3445
:10484000FE0BEA36E96E2F0EE926010EEA2212006F
:104850006AEC2AF0F350EE24006E0350EE20016E55
:104860006EEF2AF077DB05EC1AF0EFDAE66A120059
:10487000A3EC28F0020E1FC0DBFF010EDBCFE6FF2A
:10488000120068DB8DEC14F025EF27F0D950FB0FF8
:10489000F8EC29F0EE500016EE500116EE5002161C
:1048A000EE500316120097DA890EEE6E010EED6ED1
:1048B000D950120090DA8D0EEE6E010E12005C0ED1
:1048C000DBCFE9FF5D0EDBCFEAFF1200D6EC34F060
:1048D000E66A42EC34F0E5521200020E00C0DBFF43
:1048E000030E01C0DBFF1200020EDBCF00F0030E4F
:1048F000DBCF01F01200E750F4EF29F0040EF4EFE3
:1049000029F0020E1DC0DBFF030E1EC0DBFF040EEC
:104910001FC0DBFF050E20C0DBFF020E1200E126E8
:1049200001017751070D82DB800E0026000E012267
:104930001200D950060FEADAD950260F72EC2AF08D
:10494000010EDB501200E66EACEC29F038EC39F0C9
:1049500025EF27F0F90EDBCF1CF0FA0EDBCF1DF0B0
:10496000FB0EDBCF1EF0FC0EDBCF1FF012000B0E98
:1049700000C0DBFF0C0E01C0DBFF0D0E02C0DBFF31
:104980000E0E03C0DBFF12000F0EDBCF1CF0100E6B
:10499000DBCF1DF0110EDBCF1EF0120EDBCF1FF0B0
:1049A00012000F0E1CC0DBFF100E1DC0DBFF110E2E
:1049B0001EC0DBFF120E1FC0DBFF1200130EDBCF89
:1049C0001CF0140EDBCF1DF0150EDBCF1EF0160E03
:1049D000DBCF1FF01200EF50E66ED950510FF3D924
:1049E00031DC9DEF29F0BFDAEF5012001CC0DBFF75
:1049F000DBCF04F0056A066A076A120091C1E6FF80
:104A000092C1E6FF1200E76E010EE7CFDBFF120056
:104A1000D9501B0FE3EF26F0E126D9CFE9FFDACF1B
:104A2000EAFF1200D950070FEBEF26F0F90FF8EF6D
:104A300029F0040EE66EE66A120080928094808669
:104A4000828097EC37F097EC37F051EF03F00F0EC0
:104A5000E66EE66AE90EE66E000EE66EC80EE66EDB
:104A6000010E1200C8D9C8D3B6D9A60EEE6E010E3B
:104A70001200B1D9AE0EEE6E010E1200E66AD950E8
:104A8000120FE3EF26F0FB0EDBCF00F0FC0EDBCFC6
:104A900001F01200010F3ADA0C0EDB5012009E0EEC
:104AA000E66E010EE66E1200006E7851D88000545A
:104AB0001200F36E060EF3CFDBFF1200EE6E200E37
:104AC000EE6EEE6A1200DECF00F0DDCF01F01200D4
:104AD000E66A8CEC34F0E552120020EC2AF0DF6E2E
:104AE0001200140EEECFDBFF150EEECFDBFF160E1D
:104AF000EECFDBFF12006FD9490EEE6E4E0EEE6E5A
:104B00004A0EEE6E1200D950010F006ED950270FD9
:104B100048EF29F0005C000E01581200070EE66E07
:104B2000AE0EE66E4BEC3AF0E552E5521200010E85
:104B3000E66EE66EC2DBD9501200FE0EDBCFE7FF59
:104B4000F350E75EFE0EE7CFDBFF1200DBCFE6FFA0
:104B5000E66A48EF28F01BDA27EF3AF01DC004F0B0
:104B60001EC005F01FC006F020C007F01200F90EAD
:104B7000DBCF04F0FA0EDBCF05F0066A076A1200FD
:104B8000EE6E5D0E51EF28F026D9200EEE6E12006B
:104B9000DACFE6FFFC0EDBCFE6FF1200DFCFE6FF49
:104BA00020EF2AF0DBCFE6FF64EC3BF0E552120089
:104BB000E66EDBEC1FF0E5521200F36E040EF3CF4D
:104BC000DBFF1200E66E64EC3BF0E552120069DA9E
:104BD000210FEBEF26F0FFD8950EEE6E000EED6E76
:104BE0001200910EE66E010EE66E950EE66E010E57
:104BF0001200006E246EFE0EDBCF1FF0A3EF3BF021
:104C0000216ACA0E226E9A0E236E3B0E246E12008B
:104C1000216AE10E226EF50E236E050E246E12003F
:104C2000800E216E960E226E980E236E246A12005C
:104C3000400E216E420E226E0F0E236E246A120069
:104C4000226A400E236E1C0E246E8C0E256E1200FE
:104C5000080EE66EE66AC60EE66E000EE66E1200FE
:104C6000080EE66EE66AD60EE66E000EE66E1200DE
:104C7000DB50006E016A1200020EE96E010EEA6E50
:104C8000EE5079191200792B000E7A237B237C23B6
:104C9000812B1200310E926E010E936EB60E946E41
:104CA0001200230E00C0DBFF240E01C0DBFF120048
:104CB000FE0EDB04F36E040EDB50F35C12008BD8A7
:104CC0002D0EEE6EEE6E1200010EE66EFBEF26F07C
:104CD000390EDBCFE9FF3A0EDBCFEAFF1200E12607
:104CE000D950060FEBEF26F01B0EDBCFE9FF1C0EB1
:104CF000DBCFEAFF1200E126D950050FEBEF26F0DB
:104D0000180EDBCF02F0190EDBCF03F012001A0EE3
:104D1000DBCF02F01B0EDBCF03F01200140EDB6AB8
:104D2000150EDB6A160EDB6A1200180EDB6A190E0E
:104D3000DB6A1A0EDB6A1200F90EDBCFE9FFFA0E0E
:104D4000DBCFEAFF1200EECF00F0EECF01F0EECFA6
:104D500002F01200E80EEE6E030EED6E1200E66E2B
:104D600051EC3BF0E5521200100EE66ED950010FE7
:104D70001200F36E070EF3CFDBFF1200F36E030E8B
:104D8000F3CFDBFF1200CB0EE96E010EEA6E1200CC
:104D9000F36E050EF3CFDBFF1200F36E020EF3CFBE
:104DA000DBFF1200DB50F00BE8380F0B1200FE0E99
:104DB000DB5003081200020EE66ED9501200F3CF4A
:104DC000DBFFD9501200E66EDACFE6FF120095EC59
:104DD00038F0E552B2D2E96EDACFEAFF120000C035
:104DE0001CF001C01DF002C01EF003C01FF0120035
:104DF0000F0146EF21F0D9CFE6FFDACFE6FF120030
:104E0000F6EC21F04BD304C01CF005C01DF006C029
:104E10001EF007C01FF01200EE500026EE500122D7
:104E2000EE500222EE5003221200C1EC39F0BCDA3F
:104E3000D950FB0FDDDA1850EE5E0150EE5A0250E9
:104E4000EE5A0350EE5AFB0E1200F56E060EE15EAE
:104E5000F5501200BEEC21F0140F87EC21F076DA49
:104E6000020F9BEC22F072DA130F9BEF22F0FE0E82
:104E7000DBCFE6FFF2EF21F0DE6EDD6AE66A010EBF
:104E8000E66E7BDCEF50E66EE66A77DCEE52EFCF43
:104E900000F073DCEF500024FF0F6DEF21F018508D
:104EA000EE5C006E1950EE58016E1A50EE58026E0C
:104EB0001B50EE58036E1200F7DA46EF21F0E75070
:104EC0000026000EE6EF29F00250E66E8BEC21F092
:104ED00046EC21F0DEEF22F01DC022F01EC023F0D0
:104EE0001FC024F020C025F01200DF24E66E20EF62
:104EF0002AF0036AE8DA02C0EFFF12003FDAADDA07
:104F000066EF24F0E552E7CFD9FF1200006EDACF4A
:104F100001F012005BEC21F0E65212001EEC23F0CF
:104F2000050E74EC22F0060E74EC22F0070E74EC01
:104F300022F0080E74EF22F053DAD950130FA6EFC7
:104F400021F000C01DF001C01EF002C01FF003C020
:104F500020F01200EECFE6FFEECFE6FFEECFE6FF49
:104F6000EFCFE6FF1200230EDBCFE9FF240EDBCFED
:104F7000EAFF1200EF50E76EF6EC21F07BEF24F031
:104F8000BA51EA6ABB0FE96E010EEA221200100E56
:104F9000216E270E226E236A246A1200DBCFE6FF01
:104FA00081EC22F0D9501200E66E69EF21F02D0E4F
:104FB000DBCF1CF02E0EDBCF1DF02F0EDBCF1EF053
:104FC000300EDBCF1FF012000C0E00C0DBFF0D0E09
:104FD00001C0DBFF0E0E02C0DBFF0F0E03C0DBFFC4
:104FE0001200EECFE6FFEFCFE6FF81EC22F0D950C2
:104FF0001200AAEC21F0170F7CEC21F0D8EF21F081
:10500000AAEC21F01B0F7CEC21F03CEF22F0AAEC83
:1050100021F01F0F7CEC21F0E5EF21F0DF28DFEC21
:1050200023F0430EE926010EEA221200F3CF00F02E
:10503000F4CF01F01200020ED7D160EC21F069EF3D
:1050400021F04CEC21F0D9501200C1EC39F018C01D
:1050500004F019C005F01AC006F01BC007F0D950C3
:105060001200ACEC23F0010FE66E49EC22F069EC83
:1050700021F0010EACEF23F0DBCF1CF0FC0EDBCFF8
:105080001DF0FD0EDBCF1EF0FE0EDBCF1FF0120079
:10509000D950020F72EF2AF0DBCF03F0080E1F0B7E
:1050A0001200EE6EEE6AD9501200C3DCD20EE66E2C
:1050B000000EE66EF4DC69EF21F0EF50E66E010EB3
:1050C000DB50DF24C1D9010EDB2A1200006E016A19
:1050D000026A036AD950130F7CEC21F0CBEF21F068
:1050E0000B0EDBCF00F00C0EDBCF01F00D0EDBCF93
:1050F00002F00E0E1200110D0250F324006EDA5071
:10510000F420016EEBD1766B776978699FEC21F022
:10511000EF6A1200E66EF2EC21F0D950120081EC39
:1051200037F0E552E552120046EC21F0200EEF6E0A
:105130001200FE0EDBCFE6FF61EC0EF0F56E090EFD
:10514000E15EF5501200050E006E246E010EDBCFFD
:105150001FF0A3EF3BF01DC008F01EC009F01FC0F8
:105160000AF020C00BF01200E66ED950120F87EF44
:1051700021F0BEEC21F0030F87EF21F05BEC21F072
:10518000030EE12612005BEC21F0020EE126120074
:10519000F36E010EA1EF22F05BEC21F0FE0EDB04BA
:1051A0001200216E226A236A246A120094EC21F014
:1051B0007EEF24F06AEC22F019EF23F03ADC6FDC8A
:1051C000A20EE66E010E1200EAEC22F0D950020F98
:1051D000076EDACF08F01200A00E216E860E226E46
:1051E000010E236E246A1200DF28DFEC23F02F0E5D
:1051F000E926010EEA2212002CEC39F0E5529DD08E
:1052000093EC22F0A7DDB0EF23F00050F324E96E19
:10521000DA50F420EA6E1200D9D8D9501200800E6C
:10522000216EEE0E226E360E236E12009FEC21F0E0
:10523000F80EDBCFEEFFF90E12009FEC21F0FA0E14
:10524000DBCFEEFFFB0E1200FD0EDBCFE6FFFE0E06
:10525000DBCFE6FF1200DBCF05F00250E66E72EF07
:1052600021F019EC25F0CE0EE66E000EE66E12006F
:10527000EE6E3A0EEE6E200EEE6EEE6E120093ECB7
:1052800022F0E90EEE1812007EEC24F0C6EF21F0B9
:1052900029D9DF50120089EC23F0ED6ED9501200AD
:1052A000EAEC23F027EF3AF0D9CFE6FF49EF22F0FE
:1052B0005BEC21F0090EE1261200B0EC37F0E5526C
:1052C000E55212009FEC21F019EF23F0F36E070E68
:1052D000A1EF22F0F36E090EA1EF22F0E552E750A4
:1052E000EF6E12002E0EEE6EEE6A1200010EE66EEA
:1052F000E66A12008BEC21F0F8EF26F0020EE66E63
:10530000D3DF81EC22F0D9CFE6FF3DEC23F0D9507A
:10531000070F59DD060EE76E43EC25F0D0DD57DDB3
:1053200042EF21F0D950590FF1DD580EDB50F8EF64
:1053300026F072EC21F0F8EF26F0E552E552E55246
:10534000120059DDFE0EDBCFE6FF1200010EACECC1
:1053500023F0230FA6EF21F0D950010FE3EF26F041
:1053600032DD69EF21F044DDEF5030081200DBCF71
:1053700007F049DD34EC2BF080EF23F074EC22F0E1
:10538000050E1EEC23F0060E1EEF23F0000E021693
:10539000FF0E031603C002F079EF27F0B7DD010E10
:1053A000DB5026DD5DEF28F018C000F019C001F0D9
:1053B0001AC002F01BC003F01200A8DDDF50F8EFA6
:1053C00026F0ACEC23F0010FE3EF26F0012200C041
:1053D000E6FF01C0E6FF12004CEC21F037EF27F0AA
:1053E000DBCFE6FF65EF22F0E926000EEA2212008D
:1053F000E96EFF0EDA20EA6E1200DDDC330FE3DC2B
:105400005FEF24F0DB50F4DCB5DDEF502008120034
:10541000DB5046EC21F0AEDD300EEF6E1200D950BD
:10542000F8EC23F081DE070EDB2A1200D950FDECE8
:1054300023F07ADE090EDB2A1200E66AFBEF26F083
:1054400006EC35F0E5521200E66EC4EF23F0E66E8E
:1054500049EC22F0BCDC42EF21F0070E1EEC23F0F9
:10546000080E1EEF23F0EAEC22F0B6EC38F025EF40
:1054700027F0020EDB50BCDCEFCFDFFF1200DBCFEA
:1054800003F0ADDC34EF2BF0A6DCC6EC21F0B5EF79
:1054900023F0020E3FDE470FE6EF22F0060EE9266C
:1054A000000EEA22EF5012000224E96F000EDA200B
:1054B000EA6FEF5012008FDC5B0EEE6E120060ECB4
:1054C00021F0E7EF26F072EC21F046EF21F083DCCB
:1054D0000CEF27F0DBCFEAFF1BEF28F000C0E6FF60
:1054E000E66E1200026EDACF03F01200FEDC006EF0
:1054F000120000DF29EF23F0FDDE31EF23F0FADEAA
:0C55000002C0EFFF120074DC6EEF29F017
:04550C008E0E206E71
:10551000266A1D6A1C6A9AEF2AF08E0E206E1FC042
:1055200026F01D6A1C6A1FAE9AEF2AF01E6C1F1E21
:10553000E86A1F222B6AE86A1F64C3EF2AF0F00EA4
:105540001F14E866ACEF2AF01F3A1E380F0B1F2617
:105550001E38F00B1E6E2B84D8901FBEBFEF2AF0B2
:105560001E361F362B2A1FBEBFEF2AF01E361F36EF
:105570002B2A1FBEBFEF2AF01E361F362B2A2B50B8
:10558000205E31EF2BF01EC01FF01E6AE86A2B86EA
:105590001F642BEF2BF0F00E1F14E866D2EF2AF0F9
:1055A0001F3A2B84D8901FBEBFEF2AF01F362B2A3C
:1055B0001FBEBFEF2AF01F362B2A1FBEBFEF2AF0F7
:1055C0001F362B2ABFEF2AF0278027AEFF0C1F6A59
:1055D00026AE1F681FC01EF01FC01DF01FC01CF0AC
:1055E00026361F32FF0C278027AEFF0C1F6A26AE1F
:1055F0001F681FC01EF01FC01DF026361F32FF0C93
:10560000278027AEFF0C1F6A26AE1F681FC01EF042
:1056100026361F32FF0C278027AEFF0C1F6A26AEEE
:105620001F6826361F32FF0C278227AEFF0C20682A
:105630001F681E681D6826361F32FF0C278427AEA0
:10564000FF0C010E206E1F6A1E6A1D6A26361F326D
:10565000FF0C2786FF0C1F6A1E6A1D6A1C6A206ADF
:10566000000C26AE1F9E000C9E0E206E266A48EF90
:105670002BF09E0E206E1FC026F01FAE48EF2BF0C1
:10568000E86A1C6C1D1E1E1E1F1E1D221E221F22CC
:105690001F50FF0BD8B4ADEF2BF0F00BD8B486EF52
:1056A0002BF0E86A1FBE6FEF2BF0D8901C361D362A
:1056B0001E361F36E82A1FBE6BEF2BF01C361D3638
:1056C0001E361F36E82A1FBE6BEF2BF01C361D3628
:1056D0001E361F36E82A20641EEF2BF0205E27BC02
:1056E0001CAE31EF2BF0D880800E1C641D30E86AB0
:1056F0001D221E221F22D8A031EF2BF01F321E3296
:105700001D32204A14EF2BF031EF2BF01DC022F098
:105710001FC024F0D8901F34D70FF66E580EF76ACA
:10572000F722000EF86AF8220A00F5501C02F3CFA7
:105730001CF0F4CF1DF01E02F3CF1EF0F4CF1FF0CB
:105740002202F3501D26F4501E26F5502402F35079
:105750001F260800F5506BEF2BF01E501F6EFF0B3D
:10576000D8B4F6EF2BF01DC01EF01CC01DF01C6A53
:105770001F50F00BD8B4D6EF2BF0080E1FBE6BEF06
:105780002BF0D8901D361E361F36E82A1FBE6BEF51
:105790002BF01D361E361F36E82A1FBE6BEF2BF08E
:1057A0001D361E361F36E82A6BEF2BF01EC023F085
:1057B000D8901F34D70FF66E580EF76AF722000EF6
:1057C000F86AF8220A00F5501D02F3CF1DF0F4CF5D
:1057D0001EF01F02F3CF1FF02302F3501E26F450D9
:1057E0001F260800F550080F6BEF2BF01D501F6EA1
:1057F000FF0BD8B436EF2CF01CC01EF01D6A1C6ADB
:105800001F50F00BD8B41BEF2CF0100E1FBE6BEF27
:105810002BF0D8901E361F36E82A1FBE6BEF2BF0F8
:105820001E361F36E82A1FBE6BEF2BF01E361F36C2
:10583000E82A6BEF2BF01FC024F0D8901F34D70F4D
:10584000F66E580EF76AF722000EF86AF8220A0080
:10585000F5501E02F3CF1EF0F4CF1FF02402F350D8
:105860001F260800F550100F6BEF2BF01C501F6E19
:10587000FF0BD8B42BEF2BF01E6A1D6A1C6A1F5059
:10588000F00BD8B457EF2CF0180E1FBE6BEF2BF0B7
:10589000D8901F36E82A1FBE6BEF2BF01F36E82A80
:1058A0001FBE6BEF2BF01F36E82A6BEF2BF0D89062
:1058B0001F34D70FF66E580EF76AF722000EF86AFB
:1058C000F8220A00F5501F02F3CF1FF00800F55030
:1058D000180F6BEF2BF000000780064006400520F4
:1058E00005200520052004100410041004100410E5
:1058F000041004100410247E1F5024182B6E1C6A00
:10590000205025646BEF2DF024C026F0248E1F8ECE
:1059100020C02AF025C020F0E86A2A64BDEF2CF0F0
:105920002A50255ED8B45DEF2DF0070E25642BEFCD
:105930002DF0255E1DC01CF01EC01DF01FC01EF006
:105940001F6A254E5DEF2DF0256400EF2DF0255EDA
:105950001DC01CF01EC01DF01E6A254E5DEF2DF00F
:105960002564DEEF2CF0255E1DC01CF01D6A254E5F
:105970005DEF2DF02564C5EF2CF026C01FF023C08D
:105980001EF022C01DF01C6A000C030E2564D0EF2F
:105990002CF0255E1C380F0B1C6E254E5DEF2DF094
:1059A000D8901C32254E5DEF2DF0D8901C32254E3C
:1059B0005DEF2DF0D8901C325DEF2DF0030E2564C5
:1059C000EFEF2CF0255E1C380F0B1C6E1D38F00B12
:1059D0001C261D380F0B1D6E254E5DEF2DF0D89047
:1059E0001D321C32254E5DEF2DF0D8901D321C3239
:1059F000254E5DEF2DF0D8901D321C325DEF2DF05D
:105A0000030E256417EF2DF0255E1C380F0B1C6E5E
:105A10001D38F00B1C261D380F0B1D6E1E38F00BA9
:105A20001D261E380F0B1E6E254E5DEF2DF0D890F3
:105A30001E321D321C32254E5DEF2DF0D8901E32E5
:105A40001D321C32254E5DEF2DF0D8901E321D32D6
:105A50001C325DEF2DF0030E256448EF2DF0255E1E
:105A60001C380F0B1C6E1D38F00B1C261D380F0B3D
:105A70001D6E1E38F00B1D261E380F0B1E6E1F38B4
:105A8000F00B1E261F380F0B1F6E254E5DEF2DF0FD
:105A9000D8901F321E321D321C32254E5DEF2DF084
:105AA000D8901F321E321D321C32254E5DEF2DF074
:105AB000D8901F321E321D321C32216A2BAE4CEFA1
:105AC0002EF01C6C1D1E1E1E1F1EE86A1D221E22AB
:105AD0001F224CEF2EF025666FEF2DF0000C216A8F
:105AE0001FC026F01F8E248E2550205C256ED8B452
:105AF00040EF2EF0070E25640EEF2EF0255E22C03B
:105B000021F023C022F024C023F0246A254E40EF68
:105B10002EF0070E2564E3EF2DF0255E22C021F064
:105B200023C022F0236A254E40EF2EF0070E256495
:105B3000C1EF2DF0255E22C021F0226A254E40EFF4
:105B40002EF0070E2564A8EF2DF026C01FF0000CE4
:105B5000030E2564B3EF2DF0255E21380F0B216E67
:105B6000254E40EF2EF0D8902132254E40EF2EF0FA
:105B7000D8902132254E40EF2EF0D890213240EFC0
:105B80002EF0030E2564D2EF2DF0255E21380F0B89
:105B9000216E2238F00B212622380F0B226E254E63
:105BA00040EF2EF0D89022322132254E40EF2EF0D9
:105BB000D89022322132254E40EF2EF0D89022325A
:105BC000213240EF2EF0030E2564FAEF2DF0255E12
:105BD00021380F0B216E2238F00B212622380F0BB3
:105BE000226E2338F00B222623380F0B236E254E0E
:105BF00040EF2EF0D890233222322132254E40EF52
:105C00002EF0D890233222322132254E40EF2EF052
:105C1000D89023322232213240EF2EF0030E256439
:105C20002BEF2EF0255E21380F0B216E2238F00B62
:105C3000212622380F0B226E2338F00B2226233820
:105C40000F0B236E2438F00B232624380F0B246E01
:105C5000254E40EF2EF0D8902432233222322132CA
:105C6000254E40EF2EF0D8902432233222322132BA
:105C7000254E40EF2EF0D8902432233222322132AA
:105C80001C6A2BAE4CEF2EF0216C221E231E241E0C
:105C9000E86A22222322242221501C2622501D227F
:105CA00023501E2224501F222BBE63EF2EF0D8A0BB
:105CB0006FEF2BF01F321E321D321C32203E6FEF71
:105CC0002BF014EF2BF0D8B048EF2BF0E86A1C6CE7
:105CD0001D1E1E1E1F1E1D221E221F22267E48EF75
:105CE0002BF0286AE86A256429EF2BF020642BEF5B
:105CF0002BF01F502418266E1F8E248E233424343C
:105D00002B36D890E8362B36F00FF66E5F0EF76E16
:105D10002B50010BF722F86A000EF8220A00F5CF8B
:105D20001AF00A00F5CF2BF00800F5CF2AF01A5030
:105D30002A5C1A6ED89022341A02F4CFF7FF23346B
:105D40001A02F3CFE8FFF726D8B0F42A296AF750F1
:105D5000295EF4502A5AE86A2B5A1FC01AF01EC056
:105D6000F7FF1DC0F6FF1D502902F4CF1BF01E5097
:105D70002A02F4CF1DF0F3CF1CF02902F3501B26AA
:105D8000F4501C22E86A1D22F6502A02F3501B260A
:105D9000F4501C22E86A1D221F502902F3501C26D1
:105DA000F4501D221F502A021E6AE86A1E22F35078
:105DB0001D26F4501E22F6502B02F3501C26F450E0
:105DC0001D221F6AE86A1E221F22F7502B02F35081
:105DD0001D26F4501E22E86A1F221A502B02F3508F
:105DE0001E26F4501F221FBEFBEF2EF01C361D3660
:105DF0001E361F36280624C01AF023C0F7FF22C023
:105E0000F6FF22502902F4CF1BF023502A02F4CFD0
:105E100022F0F3CF21F02902F3501B26F450212267
:105E2000E86A2222F6502A02F3501B26F45021225F
:105E3000E86A222224502902F3502126F45022221B
:105E400024502A02236AE86A2322F3502226F450BF
:105E50002322F6502B02F3502126F4502222246AEA
:105E6000E86A23222422F7502B02F3502226F45012
:105E70002322E86A24221A502B02F3502326F450DE
:105E8000242224AE24BC4BEF2FF01B3621362236C1
:105E900023362436282A216C221E231E241EE86A5B
:105EA0002222232224221FC02BF01EC02AF01DC054
:105EB00029F01CC0F6FF1D502202F4CF1BF01E502B
:105EC0002102F4501B261E5022021C6AE86A1C2282
:105ED000F3501B26F4501C22F6502302F4501B26CC
:105EE0001D6AE86A1C221D2229502302F3501B263A
:105EF000F4501C22E86A1D222A502302F3501C266B
:105F0000F4501D221F502202F3501C26F4501D2273
:105F10001F5023021E6AE86A1E22F3501D26F45009
:105F20001E222B502102F3501B26F4501C22E86A3B
:105F30001D221E222B502402F4CF1FF0F3501E26E8
:105F4000E86A1F22F6502402F3501B26F4501C224C
:105F5000E86A1D221E221F2229502402F3501C260B
:105F6000F4501D22E86A1E221F222A502402F350F8
:105F70001D26F4501E22E86A1F221FBECDEF2FF00F
:105F80001C361D361E361F3628061FBECDEF2FF0DD
:105F90001C361D361E361F3628062550205E800E04
:105FA000D8A0DAEF2FF028242026D8B014EF2BF059
:105FB000DFEF2FF028242026D8A01EEF2BF027BCDF
:105FC0001CAEF4EF2FF0D880800E1C641D30E86A00
:105FD0001D221E221F22D8A0F4EF2FF01F321E32E6
:105FE0001D32204A14EF2BF026AE1F9E000CFFFF3F
:105FF00001FF04FE09FD10FC19FB23FA30F93EF8FD
:106000004EF760F674F58AF4A1F3BAF2D5F1F1F027
:106010000FF02FEF50EE73ED98ECBEEBE5EA0FEAD0
:1060200039E966E893E7C3E6F3E526E559E48EE34C
:10603000C5E2FCE136E170E0ACDFE9DE28DE68DDD8
:10604000A9DCEBDB2FDB74DABAD902D94AD894D7B2
:10605000DFD62CD679D5C7D417D468D3BAD20DD20F
:1060600061D1B7D00DD064CFBDCE17CE71CDCDCC20
:1060700029CC87CBE6CA46CAA6C908C96AC8CEC712
:1060800033C798C6FEC566C5CEC437C4A1C30CC30A
:1060900078C2E5C152C1C1C030C0A0BF11BF83BE2C
:1060A000F6BD69BDDDBC52BCC8BB3FBBB6BA2FBA9A
:1060B000A8B921B99CB817B893B710B78DB60BB66D
:1060C0008AB50AB58AB40BB48DB30FB392B216B2C7
:1060D0009BB120B1A6B02CB0B3AF3BAFC3AE4CAEBA
:1060E000D6AD60ADEBAC77AC03AC8FAB1DABABAA60
:1060F00039AAC8A958A9E8A879A80BA89CA72FA7CE
:10610000C2A656A6EAA57FA514A5AAA440A4D7A313
:106110006EA306A39FA238A2D1A16BA106A1A1A044
:106120003CA0D89F749F119FAF9E4D9EEB9D8A9D72
:10613000299DC99C699C0A9CAB9B4C9BEE9A919AA9
:10614000349AD7997B991F99C49869980E98B497F7
:106150005A970197A8965096F895A0954995F2946C
:106160009C944694F0939B934693F1929D9249920E
:10617000F691A3915091FE90AC905A900990B88FEF
:10618000688F178FC88E788E298EDA8D8C8D3E8D14
:10619000F08CA38C568C098CBC8B708B248BD98A89
:1061A0008E8A438AF889AE8964891B89D288898856
:1061B0004088F887AF8768872087D98692864C8683
:1061C0000586BF8579853485EF84AA84658421841A
:1061D000DD83998356831283CF828D824A8208821F
:1061E000C681858143810281C18081804080018098
:1061F0001C6AE86A256220642BEF2BF01F502418DC
:10620000266E255020267E0ED8A00DEF31F0205EA0
:10621000D8B014EF2BF011EF31F0205ED8A01EEFB4
:106220002BF01F8E248E1FC02BF01EC02AF01DC025
:1062300029F01D502202F4CF1BF01E502302F4CF90
:106240001DF0F3CF1CF02202F3501B26F4501C2249
:10625000E86A1D2229502302F3501B26F4501C2209
:10626000E86A1D221F502202F3501C26F4501D2202
:106270001F5023021E6AE86A1E22F3501D26F450A6
:106280001E2229502402F3501C26F4501D221F6A9E
:10629000E86A1E221F222A502402F3501D26F450C1
:1062A0001E22E86A1F222B502402F3501E26F450AF
:1062B0001F221FBE64EF31F01C361D361E361F36FE
:1062C0002006D8B41EEF2BF027BC1CAE79EF31F0BE
:1062D000D880800E1C641D30E86A1D221E221F22F9
:1062E000D8A079EF31F01F321E321D32204A14EF50
:1062F0002BF026AE1F9E000C266A24AE85EF31F0EF
:10630000236C241EE86A2422261E1FAE8DEF31F076
:106310001E6C1F1EE86A1F22261EFFEC3AF01FBEED
:106320009DEF31F026AE000C1E6C1F1EE86A1F2286
:106330001A6C1B1EE86A1B22000C26BE94EF31F07B
:106340002788FF0C1EC02AF01E502302F4CF1DF038
:10635000F3CF1CF01F502402F4CF1FF0F3CF1EF038
:106360002302F3501D26F4501E22E86A1F222A50F1
:106370002402F3501D26F4501E22E86A1F22000C4E
:10638000E86A2064000C1FC026F01F8E8E0E205C71
:10639000E8AE00EF2BF0E86C206E070E206420EFD3
:1063A00032F0205E1EC01DF01FC01EF01F6A204E7E
:1063B00049EF32F0070E2064FEEF31F0205E1EC080
:1063C0001DF01E6A204E49EF32F0030E2064F0EFFC
:1063D00031F0205E1D380F0B1D6E204E49EF32F05C
:1063E000D8901D32204E49EF32F0D8901D32204E09
:1063F00049EF32F0D8901D3249EF32F0030E20649D
:106400000FEF32F0205E1D380F0B1D6E1E38F00BA3
:106410001D261E380F0B1E6E204E49EF32F0D8900D
:106420001E321D32204E49EF32F0D8901E321D32FE
:10643000204E49EF32F0D8901E321D3249EF32F033
:10644000030E206437EF32F0205E1D380F0B1D6EF7
:106450001E38F00B1D261E380F0B1E6E1F38F00B5A
:106460001E261F380F0B1F6E204E49EF32F0D890BA
:106470001F321E321D32204E49EF32F0D8901F32AB
:106480001E321D32204E49EF32F0D8901F321E329C
:106490001D3227BC1DAE57EF32F0D880800E1D6430
:1064A0001E30E86A1E221F221FBE00EF2BF026AE10
:1064B000000C1E6C1F1EE86A1F22000C1C6AE86A92
:1064C0002064000C1FC026F01F8E1B6A9E0E205CED
:1064D000E8AEE4EF2AF0E86C206E070E20642BEFA4
:1064E00033F0205E1CC01BF01DC01CF01EC01DF050
:1064F0001FC01EF01F6A204E61EF33F02064FCEFD6
:1065000032F0205E1CC01BF01DC01CF01EC01DF030
:106510001E6A204E61EF33F02064D6EF32F0205E29
:106520001CC01BF01DC01CF01D6A204E61EF33F033
:106530002064B9EF32F0205E1CC01BF01C6A204EB4
:1065400061EF33F0030E2064ABEF32F01B380F0B1A
:106550001B6E61EF33F0D8901B32204E61EF33F0A9
:10656000D8901B32204E61EF33F0D8901B3261EF90
:1065700033F0030E2064C5EF32F0205E1C381B6E32
:106580000F0B1C6E204E61EF33F0D8901C321B3283
:10659000204E61EF33F0D8901C321B32204E61EF59
:1065A00033F0D8901C321B3261EF33F0030E2064BD
:1065B000E8EF32F0205E1C381B6E0F0B1C6E1D388E
:1065C000F00B1C261D380F0B1D6E204E61EF33F0B3
:1065D000D8901D321C321B32204E61EF33F0D89020
:1065E0001D321C321B32204E61EF33F0D8901D3229
:1065F0001C321B3261EF33F0030E206414EF33F0D2
:10660000205E1C381B6E0F0B1C6E1D38F00B1C26F9
:106610001D380F0B1D6E1E38F00B1D261E380F0B7C
:106620001E6E204E61EF33F0D8901E321D321C32A8
:106630001B32204E61EF33F0D8901E321D321C32D7
:106640001B32204E61EF33F0D8901E321D321C32C7
:106650001B3261EF33F0030E206449EF33F0205E0C
:106660001C381B6E0F0B1C6E1D38F00B1C261D38C2
:106670000F0B1D6E1E38F00B1D261E380F0B1E6EE5
:106680001F38F00B1E261F380F0B1F6E204E61EFB8
:1066900033F0D8901F321E321D321C321B32204E76
:1066A00061EF33F0D8901F321E321D321C321B3284
:1066B000204E61EF33F0D8901F321E321D321C3253
:1066C0001B3227BC1BAE71EF33F0D880800E1B64E9
:1066D0001C30E86A1C221D221E221F221FBEE4EF6E
:1066E0002AF026AE000C1C6C1D1E1E1E1F1EE86A22
:0866F0001D221E221F22000CD6
:0866F800D9CFE6FF98D1D9CFFC
:10670000E6FF95D198D9020EE126DE6ADD6ADECF7A
:1067100000F0DDCF01F0FD0EDBCF02F0FE0EDBCF8F
:1067200003F00250005C035001580AE2050EE66EC9
:1067300075EC3BF0E552DF2A010EE9E3DB2AE7D7EF
:10674000D9CFE1FF74D1D9CFE6FFE1CFD9FF020E57
:10675000E126DE6ADD6ADECF00F0DDCF01F0FD0E5E
:10676000DBCF02F0FE0EDBCF03F00250005C0350E3
:1067700001580AE200000000000000000000DF2ACB
:10678000010E01E3DB2AE7D7D9CFE1FFE552E7CFDE
:10679000D9FF120050D9FE0EDBCFE6FF85EC3BF0AF
:1067A000E552B9EC3BF0B1EC3BF00009FCE1BAEC8E
:1067B0003AF0F3CF00F0F4CF01F0040E236E246A18
:1067C000F3CF1EF0F4CF1FF07CEC31F01FC001F0CE
:1067D0001E502DD14BD94FE0030A4AE01E0A41E07A
:1067E000010A38E0030A31E0010A2AE0070A23E03F
:1067F000010A1DE0030A18E0010A14E00F0A10E084
:10680000010A0CE0030A08E0010A04E0070A39E182
:106810001DD91CD015D928D01DD926D01BD91DD0E3
:1068200015D922D00DD919D01CD9BF0E1DD0FD0EFF
:10683000FAD8EF0E19D0FD0EF6D8F346DF0E14D0BD
:10684000FD0E19D9F346F70E0FD0FAD8F114F31054
:10685000F16E17D0FD0EE7D8EF0EA214F310A26E62
:1068600010D0FFD8F3467F0E9F14F3109F6E09D00F
:10687000F8D8BF0E03D0F5D8F3467F0EF014F3100E
:10688000F06ED5D0F3D846E0030A42E0010A3EE0BC
:106890001F0A3AE0010A36E0030A32E0010A2EE05C
:1068A000070A2AE0010A26E0030A22E0010A1EE0A4
:1068B0000F0A1AE0010A16E0030A12E0010A0EE0CC
:1068C000070A0AE0010A06E0030A02E0010A23E1DE
:1068D000F28E21D0F28C1FD0F28A1DD09D801BD069
:1068E0009D8219D0A08217D09D8415D0A08013D08E
:1068F0009D8C11D09D880FD09D8A0DD09D860BD088
:10690000F28609D0A08807D09D8E05D0F28803D0EA
:10691000F08601D0F0888BD0A9D846E0030A42E087
:10692000010A3EE01F0A3AE0010A36E0030A32E0BB
:10693000010A2EE0070A2AE0010A26E0030A22E003
:10694000010A1EE00F0A1AE0010A16E0030A12E02B
:10695000010A0EE0070A0AE0010A06E0030A02E063
:10696000010A23E1F29E21D0F29C1FD0F29A1DD0A1
:106970009D901BD09D9219D0A09217D09D9415D0B8
:10698000A09013D09D9C11D09D980FD09D9A0DD0B2
:106990009D960BD0F29609D0A09807D09D9E05D069
:1069A000F29803D0F09601D0F09841D0F28C12000A
:1069B000F29C120066D8F346F346BF0E66D061D84B
:1069C000F346DF0E62D05DD8EF0E5FD034D8E652CA
:1069D000F250800B01E0010EDF6EA198FE0EDB503D
:1069E000A96EFD0EDB50A86EA69EA69CA684F29E04
:1069F000550EA76EAA0EA76EA682DF0401E1F28EE5
:106A0000A1A8FED7A198A694E55211D014D8E652B9
:106A1000FE0EDB50A96EA69EA69CA680A850DF6E37
:106A2000DF50E55204D027D8F346F3461200E55272
:106A3000E7CFD9FF1200D9CFE6FFE1CFD9FF12008F
:106A4000FD0EDB50010BF36EFE0E1200FD0E13D88F
:106A5000FB0E1200FD0EDB50010BF36EF346FD0E34
:106A60001200FD0EE0DFF346F3461200E4DFFE0EF7
:106A7000DB50120A1200DB50010BF36EF346F346B3
:106A80001200D9DFFE0E13EF35F0F114F310F16EA2
:026A9000CED75F
:0E6A9200B9B2BFB8C120B8D8B1202020202052
:106AA00000C8DDCBDFB9B2BDB320CDDDBAB3200065
:106AB0004C4544BCB7B2C120CDDDBAB3202000CBD9
:106AC000AEB3BCDECADFC0B0DDCDDDBAB300C4B842
:106AD000BCADB7C9B320BEDDC0B8202000B5CCDF47
:106AE000BCAEDDB7C9B320CDDDBAB300B7C4DEC1DB
:106AF000AEB3BEB220202020202000414C4C2043C9
:106B00004C454152202020202000CADEB0BCDEAE21
:106B1000DD20CBAEB3BCDE2000B9B2BFB8C120CA05
:106B2000DEAFB8B1AFCCDF004D454E5520455849DA
:106B3000543F202020200020C4D8AFCCDF3A4D6144
:106B4000696E2B537562200020C4D8AFCCDF3A5356
:106B500075622020202020200020CDDDBAB3C13A6C
:106B6000207878782E787825200047524E7E4F5234
:106B7000473A2020202020202020004F52477E52DC
:106B800045443A2020202020202020004D3ACADE13
:106B9000B02BBCADDDB6DD2F6B6D2B4C004D3ACA72
:106BA000DEB02BBCADDDB6DD2FCDB2B7DD00533A84
:106BB000CADEB02BBCADDDB6DD2F6B6D2B4C0053A8
:106BC0003ACADEB02BBCADDDB6DD2FCDB2B7DD00ED
:106BD000205350CADFD9BD2FBCAEB3CBD8AEB32043
:106BE00000494E4A2D54696D652FB6B2CDDEDDD811
:106BF000C20020302D3130306D20B9B2BFB8202016
:106C000020200020302D3430306D20B9B2BFB820A4
:106C100020202000B1B2C4DED8DDB8DECBAEB3BCDC
:106C2000DE20202000B7ADB3D5D8AEB3C6ADB3D803
:106C3000AEB820202000CBC2DEB9C6ADB3D8AEB806
:106C400020202020202000B9B2BDB3BCDEC4DEB3BA
:106C5000CEBEB22020202000202A56657273696FB4
:106C60006E3A20202020202A0020203A2D202020AB
:106C7000202020202B202020250020205BD6DBBCDC
:106C8000B2C3DEBDB63F205D20200020205BB8D817
:106C9000B1BCCFBCC02120205D20200020205BCDD6
:106CA000DDBAB3BCCFBCC021205D20200020205B1A
:106CB000BCDEAFBAB3BCCFBCC0215D202000202019
:106CC00020202020202020202020202020200020E4
:106CD00020202020202020202020202020202000D4
:106CE00020202020202020206D3A202020202073EA
:106CF000002020202052454144593A2020202020C5
:106D0000730020202020474F414C213A2020202092
:106D10002073004E45575245434F52443A2020209D
:106D20002020730020412F44CDDDB6DDC13A202064
:106D30002020202000454550524F4D20414C4C20F2
:106D4000434C45415200B9B2BFB8C1205BCEBFDE53
:106D5000DD5D2020202000B9B2BFB8C1205BCCB8D7
:106D6000B9DEDD5D20202000202A50432D4C494E05
:106D70004B20574149542A20002020434E4C3A4191
:106D8000504C5F45584954202000B7ADB3D5D8AE1C
:106D9000B33A202020202020202000444154453AAE
:106DA0003230202020202020202020002020204EB3
:106DB0004F572020534554555020202000001F00DD
:106DC0000000001F00001F101010101F00001F18EF
:106DD0001818181F00001F1C1C1C1C1F00001F1E61
:106DE0001E1E1E1F00001F191919191F00001F1D4C
:106DF0001D1D1D1F00001F1F1F1F1F1F000102035D
:106E00000407BADB0506070001FF02FF0304FF05C4
:106E1000060708090AFF0B0CFF0D0E0F10FF11FFEC
:066E200012FFFF1314FF36
:0A6E2600D7D8FE0EDB50080BE84041
:106E3000E840E8401F0BC8D8F346F346F3467F0E00
:106E4000DCD8040BE840E8403F0BBED8F346F346DD
:106E5000BF0ED3D8020BE8407F0BB6D8F346DF0E47
:106E6000CCD8010BB1D8EF0E8114F310816EB8D0DD
:106E7000D9CFE6FFE1CFD9FF81960000FE0EDB50AF
:106E80000F0BE66ED0DFE552FD0EDB5002E1818490
:106E900001D0819400008182000000000000000009
:106EA0008192E552E7CFD9FF120095D8E66AA0D8C3
:106EB000E66AA9D8320EE66EE66AA3EC33F0E55234
:106EC000E5528ED088D8010EE66E92D8010EE66E9D
:106ED0009AD8FE0EDB0404E0FE0EDB50020806E149
:106EE000020EE66EE66A82EC33F005D0320EE66EF4
:106EF000E66AA3EC33F0E552E55272D0010EF4EFEE
:106F000037F069D893D804E057D8FCE3DB2AFAD7E6
:106F100067D061D8E652DF6AFC0EDB50DF5C05E229
:106F20004BD801E3DB2ADF2AF7D7E55259D0140EFC
:106F30003DD8050E3BD8010E39D8010E6BD8010E95
:106F4000E66E020E6ED8010E65D82C0E4DD8080ED6
:106F50004BD80C0E49D8060E47D8010EF4EF37F087
:106F60003AD8020EE126FD0EDB0403E0400EDF6E90
:106F700001D0DF6AFE0EDB04DF26800EDF10E76E35
:106F8000010EE7CFDBFFDBCFE6FF9CDFE552D9CF79
:106F9000E1FF26D020D8FE0EDB5002E10C0E04D01B
:106FA000FE0EDB0402E10D0E1FD81AD033D8010EFD
:106FB000E66E030E11EF38F039D8E66E76DFE55253
:106FC000FD0EDB2AFE0E1200010BF36EF346F346B4
:106FD000F346F3461200D9CFE6FFE1CFD9FF120006
:106FE000E552E7CFD9FF1200E66E6CDFE5521200E2
:106FF000FE0EDB380F0B11EF38F08114F310816EA9
:10700000FE0EDB501200FE0EDBCFE6FF31DFE55255
:10701000E5521200E66EE66A82EC33F0E552E55284
:107020001200E66E25DFE552E5521200FD0EDBCFC1
:0C703000E9FFFE0EDBCFEAFFEF5012007C
:04703C00D9CFE6FFC3
:10704000DACFE6FFFA0EE3CFD9FFFB0EE3CFDAFF8C
:10705000FC0EE3CFE9FFFD0EE3CFEAFFE9CFF3FF3C
:10706000EACFF4FFF80EE35003E1F90EE35008E035
:10707000F80EE30602E2F90EE306DECFEEFFF2D7EA
:10708000FF0EE3CFDAFFE552FF0EE3CFD9FFE55263
:107090001200D9CFE6FFDACFE6FFFA0EE3CFD9FF31
:1070A000FB0EE3CFDAFFFC0EE3CFE9FFFD0EE3CFEB
:1070B000EAFFE9CFF3FFEACFF4FFE950D95CEA50E9
:1070C000DA580EE3F80EE35003E1F90EE35024E042
:1070D000F80EE30602E2F90EE306DECFEEFFF2D78A
:1070E000F80EE350D926F90EE350DA22DD52F80EFD
:1070F000E350E926F90EE350EA22ED52F80EE35090
:1071000003E1F90EE35008E0F80EE30602E2F90E9F
:10711000E306DDCFEDFFF2D7FF0EE3CFDAFFE55256
:10712000FF0EE3CFD9FFE5521200D9CFE6FFDACF49
:10713000E6FFFA0EE3CFD9FFFB0EE3CFDAFFFC0E3A
:10714000E3CFE9FFFD0EE3CFEAFFE9CFF3FFEACF9C
:10715000F4FFDECFEFFFEE66FCD7FF0EE3CFDAFFE2
:10716000E552FF0EE3CFD9FFE5521200D9CFE6FF7B
:10717000DACFE6FFFA0EE3CFD9FFFB0EE3CFDAFF5B
:10718000FC0EE3CFE9FFFD0EE3CFEAFFE9CFF3FF0B
:10719000EACFF4FFF80EE35003E1F90EE3500BE001
:1071A000F80EE30602E2F90EE306DECFEFFFEE662D
:1071B000F1D7DD52EFD7FF0EE3CFDAFFE552FF0E36
:0871C000E3CFD9FFE5521200F4
:0871C8007CD8E652006AFE0EBD
:1071D000DB50D880005408E3FE0EDB50090804E3BE
:1071E000FE0EDB50300F0AD00A0E5AD809E3FE0E0D
:1071F000DB500F0805E3FE0EDB50370FDF6E01D0CA
:10720000DF6ADF50E55262D05CD8E652300E48D8D3
:1072100008E3FE0EDB50390804E3FE0EDB50D00F0E
:1072200015D0410E3DD808E3FE0EDB50460804E3BE
:10723000FE0EDB50C90F0AD0610E32D809E3FE0EF4
:10724000DB50660805E3FE0EDB50A90FDF6E01D0B0
:10725000DF6ADF50E5523AD034D83CD801E3DB2A6C
:1072600025D801E3DB2AE552E750EF6EF6E12ED098
:1072700028D8F90EDBCF00F0DB06FA0EDBCF01F0E9
:1072800001E2DB06005001100AE024D801E3DB2A0A
:107290000DD801E3DB2AE552E750EF6EEAD716D0AE
:1072A000006EFE0EDB50D880005412000800F5502E
:1072B000E66EFD0EDBCFE9FFDB2AFE0EDBCFEAFF39
:1072C0001200D9CFE6FFE1CFD9FF1200E552E7CF98
:1072D000D9FF1200FB0EDBCFF6FFDB2AFC0EDBCF63
:0472E000F7FF1200A2
:0C72E4002A0EF66E000EF76E000EF86E1B
:1072F00001010900F550DC6F0900F550DD6F03E175
:10730000DC6701D03DD00900F550D76F0900F5507A
:10731000D86F0900F550D96F09000900F550E96EE2
:107320000900F550EA6E090009000900F550DA6F0E
:107330000900F550DB6F09000900F6CFDEF1F7CF49
:10734000DFF1F8CFE0F1D7C1F6FFD8C1F7FFD9C11F
:10735000F8FF0101DA5302E1DB5307E00900F550C1
:10736000EE6EDA07F8E2DB07F9D7DEC1F6FFDFC120
:10737000F7FFE0C1F8FF0101DC07000EDD5BBFD7BE
:027380001200F9
:0E7382001C502102F3CF18F0F4CF19F02202B4
:10739000F3501926000EF4201A6E1C502302F350ED
:1073A0001A26000EF4201B6E1C502402F3501B26DC
:1073B0001D502102F3501926F4501A22000E1B22F0
:1073C0001D502202F3501A26F4501B221D50230296
:1073D000F3501B261E502102F3501A26F4501B2294
:1073E0001E502202F3501B261F502102F3501B2671
:0273F000120089
:0E73F200D9CFE6FFE1CFD9FFAC6AAB6AFE0E41
:10740000DBB0AC88DBA202D0AC8CAB8CDBB4AC8E36
:10741000DBA602D0AB8801D0AB8ADBA802D0AC845B
:1074200001D0AC949E98DBAC02D09D8A01D09D9A8D
:107430009E9ADBAE02D09D8801D09D98FC0EDB5059
:0E744000AF6EAC8AAB8EE552E7CFD9FF1200DB
:02744E001B6AB7
:107450001A6A196A186A200EE76ED8901C361D3613
:107460001E361F36183619361A361B362150185C50
:107470002250195823501A5824501B5809E3215000
:10748000185E2250195A23501A5A24501B5A1C2A8B
:06749000E72EE4D7120014
:0A749600D9CFE6FFE1CFD9FFC26AAB
:1074A000C16AFE0EDB50C16EFE0EDB50040DF350C0
:1074B000C00BC26EFD0EDB503F0BC212FD0EDBAEE9
:1074C00003D09E9C9D8CF28CC280E552E7CFD9FF01
:0274D0001200A8
:0E74D200D9CFE6FFE1CFD9FFFE0EDB507E0BD7
:1074E000B16EB36AB26AA192FE0EDBAE02D0A08288
:1074F00001D0A092DBB2CD86DBA002D0B18E01D04C
:0C750000B19EB180E552E7CFD9FF120028
:04750C00D9CFE6FFEE
:10751000E1CFD9FFFE0EDB507E0BCD6EFE0EDBAC55
:1075200002D0CD8E01D0CD9ECF6ACE6A9E90DBAECA
:1075300002D09D8001D09D90CD80E552E7CFD9FF4C
:02754000120037
:0E754200D9CFE6FFE1CFD9FFE652F00E0001EF
:10755000FB17ABAC03D0FB91ABB0FB81ABB4FB85AD
:10756000ABB2FB87AE50DF6EDF50E552E552E7CF9E
:04757000D9FF12002D
:0C757400D9CFE6FFE1CFD9FF020EE126DF
:10758000C350DF6E010EC4CFDBFFDECF00F0DDCFD6
:1075900001F000C0F3FF01C0F4FFD9CFE1FFE552D5
:0675A000E7CFD9FF120045
:0A75A600D9CFE6FFE1CFD9FF020EB6
:1075B000E126FD0EDBCFDEFFDBCFDDFF010EDB5072
:1075C000B36EDF50B26ED9CFE1FFE552E7CFD9FFFE
:0275D0001200A7
:0E75D200D9CFE6FFE1CFD9FF020EE126FD0E74
:1075E000DBCFDEFFDBCFDDFF010EDB50CF6EDF50E8
:0E75F000CE6ED9CFE1FFE552E7CFD9FF1200F2
:0275FE001B6A06
:107600001A6A100EE76ED8901E361F361A361B36D1
:1076100023501A5C24501B5805E323501A5E245053
:0A7620001B5A1E2AE72EF0D71200B5
:06762A00D9CFE6FFE1CF1D
:10763000D9FFFE0EDB50FB0BCA6ECC6A9E92FE0E8B
:10764000DBAE02D09D8201D09D92CA84E552E7CF85
:04765000D9FF12004C
:0C7654000000000000000000000000002A
:1076600000D012001E0EE66E75EC3BF0E5521200E3
:0C7670000A0EE66E75EC3BF0E5521200CD
:04767C00D9CFE6FF7D
:10768000E1CFD9FFFE0EDB500F0BBA6EFE0EDBAE64
:1076900002D0A190A0800001FC93E552E7CFD9FF72
:0276A0001200D6
:0E76A200D9CFE6FFE1CFD9FFFE0EDB500F0B74
:1076B000BD6EFE0EDBAE02D09E949D840001FC9157
:0876C000E552E7CFD9FF1200EB
:0876C800D9CFE6FFE1CFD9FFA5
:1076D000ACAC04D0AC900001FBB3AC80FE0EDB5030
:0A76E000AD6EE552E7CFD9FF1200AE
:0676EA00FF0EE3502C6EC0
:1076F000480E01D04C0EE76EE72EFED7E76AE72E64
:0A770000FED72C2EF7D70000120070
:06770A00D9CFE6FFE1CF3C
:10771000D9FFC70EC214006EFE0EDB50380B0010EE
:0A772000C26EE552E7CFD9FF120058
:06772A0015EE00F025EE53
:1077300000F0F86A279CA68EA69C72EC39F012EC39
:0677400002F0FDD712006B
:0A7746001B6A080EE76ED8901F368C
:107750001B3624501B5C02E31B6E1F2AE72EF7D753
:02776000120015
:0A776200C250040B01E0010E1200FA
:04776C00C2909D9C8E
:02777000120005
:04777200C2841200BB
:0A7776000002376B076E060201598E
:107780006B0A6E0203026A6B0C6E0205068C6B0FAD
:107790006E020B02F26B166E020D04146C196E026F
:1077A0001101696C1E6E02FF00BE6C226E06120192
:1077B000586C206E011302466D236E070000000016
:1077C000000000000000E9030101010100000000C9
:1077D0000000000000000000006464000032FA00B5
:1077E0000000000000000000000000000000000099
:0177F0000098
:020000040020DA
:06000000313846554CFFAB
:020000040030CA
:08000000FFFAF2FEFFFFFBFF17
:00000001FF
